:1080000000000120A5340100E1090100E10901009F
:10801000E1090100E1090100E1090100000000009F
:10802000000000000000000000000000E109010065
:10803000E109010000000000E109010011860000D3
:10804000E1090100E1090100E1090100E109010084
:10805000E1090100E1090100E1090100E109010074
:10806000E1090100E1090100E1090100E109010064
:10807000E1090100E1090100E1090100E109010054
:10808000E1090100E1090100E1090100E109010044
:10809000E1090100E1090100E1090100E109010034
:1080A000E1090100F9F90000E1090100E10901001D
:1080B000E1090100E1090100E1090100E109010014
:1080C000E1090100E1090100E1090100E109010004
:1080D000E1090100E1090100E1090100E1090100F4
:1080E000E1090100E1090100E1090100E1090100E4
:1080F000E1090100E1090100E1090100E1090100D4
:10810000E1090100E1090100E1090100E1090100C3
:10811000E1090100FD1B0100E1090100E109010085
:10812000E1090100E1090100E1090100E1090100A3
:10813000E1090100E1090100E1090100E109010093
:10814000E1090100E109010075870000E109010072
:10815000E1090100E1090100E1090100E109010073
:10816000E1090100E1090100E1090100E109010063
:10817000E1090100E1090100E1090100E109010053
:08818000E1090100E109010021
:10840000FFFFFFFFFFFFFFFFFFFFFFFF7EF9FFFF03
:1084100010B5054C237833B9044B13B10448AFF3BE
:1084200000800123237010BD0086FF1F00000000A4
:10843000203A01000C4B43B10C480D4910B5AFF385
:1084400000800C48036823B910BD0A48036833B99B
:108450007047094B002BF7D0BDE810401847064B7A
:10846000002BF5D0184700BF00000000203A0100A3
:108470000486FF1F7C85FF1F0000000080F3118829
:1084800070472F4B41F238015A5842F478525A50F3
:108490002C4A927902F00C020C2A4FD041F244028D
:1084A0002949995003F558339A78110748BF9A78AB
:1084B000264944BF42F008029A70214B41F244021F
:1084C000995041F204015A5842F4803242F0C002FD
:1084D0005A501A6842F440221A6003F5E833242205
:1084E0005A701B4A80211170A2221A70DA7802F0A9
:1084F0001F02DA7003221A7100225A719A799207C8
:10850000FCD59A79D006FCD40E4B19469A7902F024
:108510000C02082AFAD140225A718B7903F00C031D
:10852000082BFAD1074B1A4699794906FCD5222126
:108530001970937903F00C030C2BFAD1704700BF2C
:1085400000700440004006400000330100001301A9
:1085500000500640284B5A7902F0E0025A711A790D
:1085600002F0F8021A71254A136843F004031360FD
:10857000234A136823F0784323F001031360214B4F
:108580001A7802F08C0242F050021A705A7802F007
:108590009C0242F040025A709A7802F0E6029A7009
:1085A000194A0023137083F31188184B012283F8B2
:1085B000182383F81923022283F83C2383F83D23F0
:1085C00083F84B2383F84C2383F84D2383F84E2301
:1085D00083F84F23032283F81F2383F8212383F892
:1085E000232383F8252383F84223042283F83B23A3
:1085F000052283F83523704700F00740408004408F
:1086000000D0004000D0074000E0074000E100E05B
:108610000F4A1368013313600E4A13680133136065
:108620000D4B1A683AB11A68013A1A601B6813B9FF
:108630000A4B01221A700A4B1A6812B11A68013AE1
:108640001A60084B1A6812B11A68013A1A6070472A
:108650001C86FF1FF8080020A4030020A0030020B0
:10866000A803002064070020024B034A5A60072237
:108670001A60704710E000E000770100014B1868B5
:10868000704700BF1C86FF1F1449154B41F228029A
:108690000B2888BF002010B553F82030114CB4FBD4
:1086A000F3F48B5843F480638B500F4B4FF44072BC
:1086B0009A634220DA6308F0B1F90C4B0022DA70B9
:1086C0009A709A71DA725A71C4F30422E4B21A7081
:1086D0005C70DA7842F02C02DA7010BD0070044051
:1086E00050370100C0C62D0000B0044000A00E406D
:1086F000094A136851680133202B08BF00238B42BD
:1087000008D01168114408721360044AD37843F00A
:108710008003D370704700BF2086FF1F00A00E406B
:108720000A4B996ADA6A91420DD09A6A511C1A442E
:10873000996292F8302002709A6A202A01D10022B0
:108740009A62012070470020704700BF2086FF1FFB
:10875000044B1A7802F0FF0012B100221A700120B7
:10876000704700BFA0030020014B1865704700BF91
:108770002086FF1F30B526480179C9B28C0617D56F
:10878000244BDA6A9C6A0132202A08BF0022A242E6
:108790001BBFDC6AC579C27918191EBFEDB280F81B
:1087A0003050DA621C4A052010601A6D1B4B1A60AB
:1087B0004A0608D51A4B4FF480529A60144AD3786F
:1087C00003F0BF03D3700B061BD5144B1868C0B958
:1087D000104B19685A68914214D0114A4FF48051D5
:1087E00051605A68511C1A445960117A084AC9B23A
:1087F000D1715968202908BF5860D37843F04003ED
:10880000D37030BD024AD37803F07F03F8E700BF8E
:1088100000A00E402086FF1FA4030020A803002014
:1088200080F00F4062B67047FFF7FCBF72B670472A
:10883000FFF7FCBF4FF0E02318B1034AC3F80C2D3B
:108840007047024AFAE700BF0400FA050100FA0582
:10885000F7B5464C4649474D474E4FF480730622C4
:108860006360A36023618A6010224A601E224A610D
:10887000424A53629364D3644FF400226A61AA604F
:108880003F4A4FF4907050621363936402F53422B0
:1088900080324FF4905090604FF48020506000F58B
:1088A00090505061374A40F2031010605060906061
:1088B000D060106150619061D06133480022426104
:1088C0003248036143618361836600F5322000F51D
:1088D000807086604661082623601046E360B446D7
:1088E0000A242B4617468E46C1F804C00197019D05
:1088F000B5F57A7F30D3DEF810508E60ED0748BFB3
:1089000001300197019DB5F57A7F29D3DEF810502B
:10891000ED0758BF0132013CE6D10A281C4923D19A
:108920000A2A21D101220A70104A4FF4E061116035
:10893000D16002F53622102191604FF400225A6076
:108940000E4A4FF48071116001225A605A6942F058
:1089500001025A6103B0F0BD019D01350195C6E7E2
:10896000019D01350195CDE70022DCE70090044030
:1089700000F00F4040F00F407000000400A00440E1
:1089800000B0044000C00440C0F00F4000D00440DC
:1089900008040020F7B5104B1B78D3B10F4B104DD6
:1089A00002210F46042000241E469F605860019457
:1089B000019AAA4209D97160B0600194019AAA4251
:1089C000F3D8019A01320192F8E7019A013201923B
:1089D000EEE703B0F0BD00BF0804002000F00F4038
:1089E0001FA10700032806D8DFE800F00206080AE6
:1089F0001022054B5A6070472022FAE74022F8E720
:108A00004FF08062F5E700BF00F10F40032806D861
:108A1000DFE800F00206080A1022054B9A60704752
:108A20002022FAE74022F8E74FF08062F5E700BF26
:108A300000F10F4038B500210446012505FA01F385
:108A40002342C8B205D0FFF7CDFF01312029F5D16F
:108A500038BDFFF7DBFFF8E708B5032813D8DFE8D8
:108A600000F0020C0E10002006F050FE43F27C03D2
:108A7000984294BF0020012008BD0120F4E70220A5
:108A8000F2E70320F0E7002008BD032817D8DFE84D
:108A900000F002070C110B4B1868C0F30010704770
:108AA000084B1868C0F340107047064B1868C0F3B5
:108AB00080107047034B1868C0F380607047002037
:108AC000704700BF00F10F4070B500242546012615
:108AD000E0B2FFF7C1FF10B106FA04F31D43013401
:108AE0001F2CF5D1284670BD024B1869C043C0B297
:108AF000704700BFC0F00F4037B50446FFF7BEFD1A
:108B00000546FFF7BBFD401B0028B8BF40420128C7
:108B1000F7DD0020012C8DF804008DF8050010D041
:108B200007D3022C11D0030648BF60F0FF0003B04A
:108B300030BD022201A9902007F01AF89DF8040028
:108B4000F1E7022201A99220F6E7224601A994202A
:108B5000F2E708B5082006F0D9FD5E281AD91D4BAA
:108B60001A780AB901221A70082006F0CFFDA92848
:108B700018D9194B1B78ABB9184B4FF400725A60D7
:108B80000C2006F0C3FD6E281AD9144B4FF4802236
:108B90005A6008BD082006F0B9FD5428E4D8002228
:108BA0000C4BE0E7082006F0B1FD952803D90A4BED
:108BB0001B78002BE4D0094B4FF400729A60DFE77A
:108BC0000C2006F0A3FD4F289EBF044B4FF48022DB
:108BD0009A6008BD7486FF1FE303002080F00F40F9
:108BE000034B1878013801288CBF00200120704702
:108BF0007486FF1F034B1878012806BF02221A70E3
:108C0000002070477486FF1FC0B207F0CBBCC0B213
:108C100007F0B6BC08B509F015FE08F0D3F808F067
:108C200083F8BDE8084009F08FBE38B5054607F067
:108C3000D1FF08280AD900242819013408F04AF87D
:108C4000092CF9D108F07AF8012038BD002038BD90
:108C5000092107F0DFBF002008F06CBA2249234841
:108C600041F23C028B5843F440538B50204B01217E
:108C700019601A6802431A601E4ADA601A61DA6AD9
:108C800042F08052DA621A6822F001021A601A6811
:108C900022F000621A60184A4FF4007313605360A8
:108CA0009360D360136153619361D361A2F5F03295
:108CB00011601168014311601049D16001F5200174
:108CC0001161D16A41F08051D162116821F0010136
:108CD0001160116821F00061116002F5E8329362C1
:108CE000D36213645364704700700440000C1F800B
:108CF00000C002400100003E00B004400400513EAC
:108D0000FF2810B54FEA004323D82B4C03F47C1303
:108D10008AB141F000610B436363E36A002BFCDA24
:108D2000254BDA6AD000FCD5986BDA6A42F0104223
:108D3000C0B2DA6210BD41F000410B436363E36AE5
:108D4000002BFCDAA06BE36A43F01043C0B2E3628D
:108D500010BDB0F5007F17D2184C03F47C135AB144
:108D600041F000610B436363E36A002BFCDA134BB1
:108D7000DA6AD100FCD5D7E741F000410B436363C9
:108D8000E36A002BFCDADDE70D4C03F47C135AB1E7
:108D900041F000610B436363E36A002BFCDA084B8C
:108DA000DA6AD200FCD5BFE741F000410B436363B0
:108DB000E36A002BFCDAC5E700C0024000D00240A5
:108DC00000C00A4010B5FFF759FC0446FFF756FCF7
:108DD000001B0028B8BF40420628F7DD10BD07B5CC
:108DE000030A8DF805008DF80610032201A9A020C2
:108DF0008DF8043006F096FEFFF7E4FF03B05DF84F
:108E000004FBF0B5154600228BB00F461446AC4269
:108E100001D10BB0F0BD0AAB1344395D03F8221C3D
:108E2000531CC618F10602D0691E8C420DD1030AEC
:108E30008DF80500033201A9A0208DF8043006F05A
:108E400071FEFFF7BFFF3046002301341A46DEE70C
:108E500030B50B4D85B02B68002BFCD1030A0224E2
:108E60008DF80C3003AB8DF80D00009422461946A6
:108E7000A02006F0A3FE9DF80C002C6005B030BDCC
:108E8000640700201FB50A4C0B4621680029FCD15D
:108E9000010A8DF80C108DF80D00009203A9022232
:108EA000A02006F08BFE0223236004B010BD00BF9B
:108EB0006407002030B4C0EBC000074C0D6825509B
:108EC00022188C8894808B79937100F5B04007222A
:108ED00030BCFFF796BF00BF7586FF1F054BC0EB88
:108EE000C000184403680B6083888B8083798B7182
:108EF000704700BF7586FF1F30B500238BB001ADF2
:108F00001A465A550133222BFBD14FF4B044230AA1
:108F10008DF8054022222946A02020348DF8043007
:108F200006F000FEFFF74EFFB4F5484FEFD10B49B6
:108F300000220C461346C2EBC20020440132B2F5B7
:108F4000805F0B704B708B70C370037143718371C2
:108F500001F10701EFD10BB030BD00BF7586FF1FD7
:108F600013B50C46C0EBC0000722694600F5B040BF
:108F7000FFF788FF9DF8002023789A4212D19DF8D0
:108F8000012063789A420DD19DF80220A3789A427D
:108F900008D1DDF80300D4F80330C31A5842584111
:108FA00002B010BD0020FBE77047F0B545F2FF703E
:108FB00085B0FFF74DFF552803D13E4B1B78002BA2
:108FC00043D0002145F2FF70FFF709FFFFF794FF40
:108FD00040223949394F3A4E0020FFF712FF4FF433
:108FE000B7654024204680223946FFF70AFF8034C7
:108FF000284660223146FFF704FFB4F5E07F05F113
:109000006005EFD104AD002345F8043D4FF4D3646F
:1090100040F678062046042229460434FFF7F1FE84
:10902000B442F7D1002303934FF4FF6440F6D8060F
:109030002046042229460434FFF7E3FEB442F7D168
:10904000552145F2FF70FFF7CAFE40221A491D4D17
:109050001B4E0020FFF716FF80221B494020FFF720
:1090600011FF80221949C020FFF70CFF8022184908
:109070004FF4A070FFF706FF002428196022314644
:10908000603409F075FCB4F5907FF6D158238DF863
:10909000083000238DF80930FFF794FE4FF4E043C9
:1090A000009302220B4B02A9A02006F087FD05B019
:1090B000F0BD00BF080400200C80FF1FE037010056
:1090C00080370100B405002030040020B0040020E7
:1090D000300500207586FF1F044B9B78022B044B44
:1090E0008CBF042203221A70704700BF680700205B
:1090F000FC0800200F4A1048002330B519461370B1
:109100005370141D4FF0FF3544F82350C154013300
:109110002F2BF9D1094B82F8C0101960084B82F847
:10912000CC101960074BC2F8C410C2F8C8101960FF
:1091300030BD00BF78F6FF1F31070020E80800208F
:10914000040900207007002038B5014C637801E065
:1091500068070020FF2B00F27585DFE813F00F028F
:1091600025024E025B0262026E0276027E028602D7
:109170008F0295029E02A702BB02CF02D702E40231
:10918000EC02F4020103090316031E0326032E0357
:1091900036033E0345034C036003730573057305F3
:1091A000690370037703730573057305730573050E
:1091B00073057305730573057305730573057305EF
:1091C00073058003730573057305730573057305D4
:1091D00073057305730573057305730573057305CF
:1091E00073057305730573057305730573057305BF
:1091F00073057305730573057305730573057305AF
:10920000730573057305730573057305730573059E
:10921000730573057305730573057305730573058E
:10922000730573057305730573057305730573057E
:109230007305730573058F039803A103AA03B30392
:10924000BC03C503CE03D703E003E903F203FB032A
:10925000040473050D0414041D0426042F043704AC
:109260003E04730546044D0454045A047305630414
:109270006D04770473058004730573057305730526
:10928000730573057305730573057305730573051E
:10929000730573057305730573057305730573050E
:1092A0007305000115011B01210131014101470135
:1092B0004D01530159015F0165016B017305730590
:1092C0007101730577017D01830191017305AD0182
:1092D000B301B901D501DB01E101E801FD010302A0
:1092E0008B049304A004AE04B504C904DE04EA04AC
:1092F000F204F804730509027305010509051E054A
:109300002505320573053B0544054D0573057305B9
:10931000730573057305730573057305730573058D
:10932000730573057305730573057305730573057D
:10933000730573057305730573057305730573056D
:10934000730573057305730573057305730573055D
:109350005605730560057305730573056A05A078E6
:1093600006F025FF964B5860964B1B785BB1944BEB
:109370005A68954B1A60954B002A40F068841A6829
:1093800042F008021A6038BDA07806F03AFF8C4B14
:109390005860E9E7A07806F042FF894B5860E3E7A0
:1093A000A078874D06F02DFFA37820B9184606F067
:1093B00050FF6860D8E7184606F038FF6860D3E7CA
:1093C000A0787F4D06F01DFFA37820B9184606F05F
:1093D000E7FE6860C8E7184606F034FF6860C3E738
:1093E000A07806F0CBFE764B5860BDE7A07806F07B
:1093F000DBFF734B5860B7E7A07806F0B5FF704B02
:109400005860B1E7A07806F0B6FF6D4B5860ABE747
:10941000A07806F0A2FF6A4B5860A5E7A07806F096
:10942000B1FF674B58609FE7A07806F0C4FF644B1C
:10943000586099E7A07806F0ACFF614B586093E75D
:10944000A07806F0C9FE5E4B58608DE7A07806F064
:1094500002FF5B4B586087E7A3785D4AD25C584BAC
:109460005A6081E7A1785B4B5B4A03EBC11302EBC7
:1094700081021869D2F8D0209047514B586073E7A9
:109480001421A0784E4D06F027FD0028D5BF6FF0BF
:109490007F43524B6B6093FBF0F0A2784D4BC8BFFB
:1094A000686003EBC2131B7E002B7FF45DAF68681E
:1094B00007F08DFA686057E7A07806F0A9FE404BE8
:1094C000586051E7A07806F079FE3D4B58604BE7B5
:1094D0001321A0783A4D06F0FFFC0028D5BF6FF0AD
:1094E0007F433E4B6B6093FBF0F0A278394BC8BFD3
:1094F000686003EBC2131B7E002B7FF435AF6868F6
:1095000007F065FA68602FE7A07806F0DFFF2C4BC4
:10951000586029E7A07806F0E0FF294B586023E760
:109520007121A07806F0D8FC254B58601CE700217B
:10953000A07806F0D1FC42070AD56F21A07806F08A
:10954000CBFC10F4804F03D01D4B01225A600BE777
:109550001B4B00225A6007E7A07806F0B0FF184BBB
:10956000586001E7A07806F0A3FF154B5860FBE6B2
:10957000A07806F08FFF124B5860F5E6A078104DEA
:1095800004F0BCFEA378372120B9184607F06AF82A
:109590006860E9E6184607F065F8A278104B53F8C2
:1095A0002230C01A6860DFE6A0780E4A044D6023BE
:1095B00043432121D35CBBB907F054F86860D3E67C
:1095C000FC080020F7080020E808002070070020B1
:1095D000E00300203004002078F6FF1F0024F40090
:1095E000D4030020B405002007F03CF8A2789F4B7C
:1095F00053F82230C01A6860B6E6A0789C4B03EBA3
:1096000080032421D3F8D04007F02CF8A047994BD1
:109610005860A9E62221A07807F024F8954B5860FD
:10962000A2E6A278924B03EB8203D3F8D020D3F8C2
:10963000DC0090478F4B586096E6A2788E4B03EB88
:10964000C2139A6A8B4B5A608EE6A2788A4B03EB60
:10965000C2135A7A874B5A6086E6A278864B03EB90
:10966000C2139A7A834B5A607EE60F21A07806F0E7
:10967000F9FF804B00F00100586075E6A07807F014
:1096800093F97C4B58606FE60F21A07806F0EAFF53
:10969000784BC0F30020586066E60F21A07806F0F2
:1096A000E1FF744BC0F3C01058605DE60121A07863
:1096B00006F0D8FF830741BF6E4A536843F00103A9
:1096C000536005077FF550AE6A4A536843F00203C2
:1096D000536049E60121A07806F0C4FFC40741BFEA
:1096E000644A536843F00103536041077FF53CAE81
:1096F000604A536843F00203536035E6A2785E4B3C
:1097000003EBC213DA7D5B4B5A602DE6A078584B11
:1097100003EB80032521D3F8D04006F0A3FFA04738
:10972000544B586020E6A278534B03EBC2131A6BDC
:10973000504B5A6018E6A2784F4B03EBC213DA6A1B
:109740004C4B5A6010E6A078494B03EB800327216D
:10975000D3F8D04006F086FFA047464B586003E69A
:10976000A278454B03EBC2135A6B424B5A60FBE5A0
:10977000A0783F4B03EB80032621D3F8D04006F0BE
:1097800071FFA0473B4B5860EEE5A2783A4B03EBE4
:10979000C2139A6B374B5A60E6E5A278364B03EB5F
:1097A000C213DA6B334B5A60DEE5A278324B03EB1F
:1097B000C2131A6C2F4B5A60D6E5A2782E4B03EBDE
:1097C000C2135A6C2B4B5A60CEE5A2782A4B03EB9E
:1097D000C2139A6C274B5A60C6E53321A07806F075
:1097E00041FF244B5860BFE53421A07806F03AFFD2
:1097F000204B5860B8E50121A07806F033FF4206FF
:1098000041BF1C4A536843F00103536003067FF5D0
:10981000ABAD184A536843F002035360A4E501213D
:10982000A07806F01FFF134BC0F3012058609BE5A2
:109830000121A07806F016FF10F0100F83E6012139
:10984000A07806F00FFF10F0200F7CE6A2780A4BFC
:1098500003EBC21393F84F20064B5A6084E5A078BF
:1098600005F01AF9034B58607EE500BFD4030020D1
:1098700078F6FF1FFC08002030040020964AA378E9
:10988000602101FB03235A68944B5A606CE5924AAD
:10989000A378602101FB03239A68904B5A6063E52B
:1098A0008D4AA378602101FB03231A7B8B4B5A60FE
:1098B0005AE5894AA378602101FB0323DA89874BA3
:1098C0005A6051E5844AA378602101FB03231A6999
:1098D000824B5A6048E5804AA378602101FB03234C
:1098E0001A7D7E4B5A603FE57B4AA378602101FBDD
:1098F00003235A7D794B5A6036E5774AA378602175
:1099000001FB03231A6A754B5A602DE5724AA3784E
:10991000602101FB03235A6A704B5A6024E56E4AAA
:10992000A378602101FB03239A6A6C4B5A601BE504
:10993000694AA378602101FB0323DA6A674B5A6006
:1099400012E5654AA378602101FB03231A6B634B80
:109950005A6009E5604AA378602101FB03239A69F4
:109960005E4B5A6000E55C4AA378602101FB03234B
:10997000DA695A4B5A60F7E47C21A07806F072FE4F
:10998000564B5860F0E4544AA378602101FB03234E
:109990005A6B524B5A60E7E44F4AA378602101FBAF
:1099A00003239A6B4D4B5A60DEE44B4AA378602147
:1099B00001FB03239A7D494B5A60D5E4A278484BBA
:1099C000134493F8E820454B5A60CDE42021A07859
:1099D00006F048FE414B5860C6E4A278602353432A
:1099E0003D4AD25C3D4B5A60BEE46621A07806F049
:1099F00039FE3A4B5860B7E46521A07806F032FE94
:109A0000364B5860B0E4A07804F078FC334B5860D3
:109A1000AAE4314AA378602101FB0323DA6B2F4BC0
:109A20005A60A1E42C4AA378602101FB032393F838
:109A300040202A4B5A6097E4274AA378602101FB13
:109A4000032393F84120254B5A608DE4224AA378E2
:109A5000602101FB03235A6C204B5A6084E40A21E5
:109A6000A07806F0FFFD1D4B00F00F00C0F10800CC
:109A7000586079E4A2781B4B03EBC2131A7A174B98
:109A80005A6071E4A278164BD10103EB8203154AA8
:109A9000D3F8D03050589847104B586064E4A17800
:109AA000104B0F4A03EBC11302EB81025868D2F846
:109AB000D0209047094B586056E40B4BA27853F8DE
:109AC0002220064B5A604FE4084BA27853F822201C
:109AD000024B5A6048E400BFB4050020FC08002097
:109AE00078F6FF1F30040020C0030020D4060020B9
:109AF000A078594A594D602343433621D35C1BB9A2
:109B000006F0B0FD68602FE406F0ACFDA278544B7F
:109B100053F82230C01A686026E45121A07806F07C
:109B2000A1FDA2784F4B53F82230C01A4B4B58601E
:109B30001AE4A2784C4B03EBC2139A7D474B5A6050
:109B400012E4A07806F0F6F8444B58600CE4A278D2
:109B5000454B03EBC213B3F84C20404B5A6003E46F
:109B6000424BA27853F822203C4B5A60FFF7FCBBD3
:109B7000A2783F49394B8C5C002058600CB101241D
:109B80005C6088543B49885C18B1586840F002001A
:109B9000586000238B54FFF7E7BBA378364AD25CAA
:109BA0002E4B5A60FFF7E0BB5021A07806F05AFD1B
:109BB000A2782C4B53F82230C01A284B5860FFF77C
:109BC000D3BBA278284B03EBC213DA69234B5A604C
:109BD000FFF7CABBA278244B03EBC2131A6A1F4BD0
:109BE0005A60FFF7C1BBA2781F4B03EBC2135A6A3E
:109BF0001A4B5A60FFF7B8BBA2781B4B03EBC2139A
:109C00009A8A164B5A60FFF7AFBBA278164B03EB4C
:109C1000C21393F84E20114B5A60FFF7A5BB0021E9
:109C2000A07806F01FFD0D4BC0F300705860FFF7E1
:109C30009BBBA2780C4B03EBC2131A7E074B5A60F6
:109C4000FFF792BB054B03221A70FFF78DBB1A6812
:109C500022F00802FFF796BBB4050020FC080020A4
:109C6000D4030020EC03002030040020FC0300207B
:109C700028040020E40300202B04002038B5C04A4B
:109C800090780228144600F0F080032800F0F48059
:109C9000002840F0D18153784D2B00F0A2803AD8B3
:109CA000452B7AD016D8412B6ED004D8402B64D0E7
:109CB0000322B44B5FE0422B6AD0442BF8D1B24967
:109CC000D2F8033041F81C3F04221C20BDE8384084
:109CD000FFF797B8492B6DD014D8462B62D0472B8D
:109CE000E6D1A94DD2F803302946042241F8083FB5
:109CF0000820FFF786F82A8A29896879BDE8384064
:109D000005F038BD4B2B61D04C2BD1D19E4BD17877
:109D10009970022034E0542B00F0848018D8512B25
:109D20006BD008D84F2B61D0502BC1D1964BD17836
:109D30009975162024E0522B6CD0532BB8D1924D3C
:109D4000D2F803302946042241F8103F1020D0E712
:109D5000842B7FD009D8552B70D0832BA8D18B4B67
:109D6000D2F80320C3F8EC2038BD852B77D0FF2B29
:109D70009ED1D278864B1A7038BDD17845F2FF70EB
:109D8000BDE83840FFF72BB87F4BD1781970F7E763
:109D90007D4BD17859700120F2E77B4BD178597116
:109DA0000520EDE77849D2F8033041F80C3F042252
:109DB0000C208BE7D278744B1AB9DA75D97D17204D
:109DC000DEE770490122DA754A60F7E76E4CD17818
:109DD000E1700320FFF703F8E078BDE83840FEF7B4
:109DE000C3BC694BD17859751520C9E7D2F8031067
:109DF000654BC9B259761920C2E7634D2A7DD20757
:109E000004D5E378DB0701D4FFF776F8E17829750C
:109E10001420B5E75C49D2F8033041F8203F042212
:109E2000202053E7D2F80330012B00F20581564978
:109E3000D37801F81A3F01221A2047E7D2F80330FD
:109E4000012B00F2F9805049D37801F81B3F012221
:109E50001B203BE74F4BD2F803201A6038BD4B4B19
:109E6000D2F80320C3F8F02038BD51784A4BD2F81D
:109E7000032043F8212038BD53782E2B3FF618AF2E
:109E800001A252F823F000BF459F0000599F000037
:109E90006D9F0000B19C0000B19C0000B19C0000CF
:109EA000B19C0000B19C0000B19C0000799D0000B5
:109EB000799D0000799D0000B19C0000B19C0000DC
:109EC000B19C0000B19C0000B19C0000B19C00005E
:109ED000B19C0000B19C0000B19C0000B19C00004E
:109EE000B19C0000B19C0000B19C0000B19C00003E
:109EF000B19C0000A19F0000AD9F0000B99F000031
:109F0000C59F0000D19F0000DD9F0000B19C0000B4
:109F1000B19C0000B19C0000B19C0000B19C00000D
:109F2000B19C0000E99F0000F39F0000FD9F00002E
:109F300007A0000011A000001BA0000025A0000049
:109F40002FA00000154BD4F803201A60FEF796FBF3
:109F50000E4BC3F8F40038BD104BD4F803205A6000
:109F6000FEF78CFB094BC3F8F80038BD0B4BD4F857
:109F700003209A60FEF782FB044BC3F8FC0038BD57
:109F800068070020FC0800200C80FF1F78F6FF1FE8
:109F9000F6080020F808002008090020E00600204C
:109FA000D4F80330254ADBB2137638BDD4F8033039
:109FB000224ADBB2D37638BDD4F803301F4ADBB275
:109FC000537638BDD4F803301C4ADBB2137738BD62
:109FD000D4F80330194ADBB2937638BDD4F8033095
:109FE000164ADBB2537738BD144BD4F803201A62FB
:109FF00038BD124BD4F803205A6238BD0F4BD4F849
:10A0000003209A6238BD0D4BD4F80320DA6238BDC4
:10A010000A4BD4F803201A6338BD084BD4F8032048
:10A020005A6338BD054BD4F803209A6338BD034BFF
:10A03000D4F80320DA6338BD04223AE6E0060020B3
:10A040002DE9F84F2D4FBB78022B52D82C4EDFF85C
:10A05000C0A0DFF8C0B00025B046BB78ECB2A34288
:10A0600008D008EBC31393F84E30CBB396F84E20CC
:10A070009A4235D1204604F077F9224A00234FF066
:10A080000109AB5405F80A304FF0006205F80B9057
:10A090004946204606F026FBF27D42BB4A46202177
:10A0A000204606F0B9FA184BD7F8030053F82530CC
:10A0B000984724210246204606F0AEFA4FF080521F
:10A0C0000721204606F00EFB4FF0006207212046D4
:10A0D00006F016FB4FF000620121204606F010FB4F
:10A0E0000135032D06F18006B7D1BDE8F88F0222B5
:10A0F000D5E7064B04221A70BDE8F88F68070020E8
:10A10000300400202804002078F7FF1FFC080020FE
:10A11000E4030020E70300202DE9F84F2E4FBB7821
:10A12000022B53D82D4EDFF8C4A0DFF8C4B00025B1
:10A13000B046BB78ECB2A34208D008EBC31393F847
:10A140004E30D3B396F84E209A4236D1204604F0D2
:10A150000BF9234A00234FF00109AB5405F80A30EC
:10A160004FF0006205F80B904946204606F0BAFA17
:10A17000F27D4ABB4A462021204606F04DFAD7F828
:10A180000300184B404253F82530984724210246DB
:10A19000204606F041FA4FF080520721204606F093
:10A1A000A1FA4FF000620721204606F0A9FA4FF00D
:10A1B00000620121204606F0A3FA0135032D06F1C5
:10A1C0008006B6D1BDE8F88F0222D4E7064B042200
:10A1D0001A70BDE8F88F00BF680700203004002027
:10A1E0002804002078F7FF1FFC080020E40300206B
:10A1F000E70300202DE9F047184E194FDFF864906F
:10A200000025B0464FF0010ABB78ECB2A34208D05B
:10A2100008EBC31393F84E30BBB196F84E209A4228
:10A2200013D1204605F066F9F37D05F809A09BB926
:10A2300001222021204606F0EFF9204600222421A9
:10A2400006F0EAF9204604F08FF80135032D06F1F7
:10A250008006D9D1BDE8F0870222EAE73004002069
:10A2600068070020E7030020014B93F80C017047BA
:10A2700078F6FF1FF8B5664E664AC701F519044621
:10A28000A96A91420CD8EB6A934209D82B6B93428E
:10A2900006D86B6B934203D8AB6B934240F281803C
:10A2A0003E4402220021204606F01CFAD6ED0A7A2E
:10A2B000F8EE677A17EE900A08F058FD0022564B28
:10A2C00008F0A8FD50A3D3E9002308F0CDFE08F064
:10A2D000B3FF28210246204606F09EF9D6ED0B7A00
:10A2E000F8EE677A17EE900A08F040FD00224A4B1C
:10A2F00008F090FD44A3D3E9002308F0B5FE08F070
:10A300009BFF29210246204606F086F9D6ED0C7AFD
:10A31000F8EE677A17EE900A08F028FD00223E4B0F
:10A3200008F078FD38A3D3E9002308F09DFE08F07B
:10A3300083FF2A210246204606F06EF9D6ED0D7AFB
:10A34000F8EE677A17EE900A08F010FD0022324B03
:10A3500008F060FD2CA3D3E9002308F085FE08F087
:10A360006BFF2B210246204606F056F9B06B07EE34
:10A37000900AF8EE677A17EE900A08F0F7FC0022D0
:10A38000254B08F047FD20A3D3E9002308F06CFE1D
:10A3900008F052FF02462C212046BDE8F84006F0A6
:10A3A0003BB91E4E06EB84060222002106F0A8F9F6
:10A3B000D6F81031A86A984728210246204606F0B0
:10A3C0002BF9D6F81031E86A984729210246204631
:10A3D00006F022F9D6F81031286B98472A21024658
:10A3E000204606F019F9D6F81031686B98472B21F2
:10A3F0000246204606F010F9D6F81031A86B9847AF
:10A40000C8E700BFAFF30080000000A2941AED423D
:10A4100030040020FFFF3F000000404278F6FF1F9D
:10A420002DE9F74F544B03EBC013824693F84F408E
:10A43000DA6B1E6CA4FB02895A6C9B6CA4FB0212A3
:10A44000CDE900126FF07F42A4FB06674245A4FBF2
:10A4500003454FF0000373EB09010CDBB24273EBD1
:10A46000070108DBDDE900BC5A4573EB0C0102DB98
:10A47000A242AB4163DA04220021504606F032F9D1
:10A480004946404608F0D0FF08F070FC36A3D3E9F7
:10A49000002308F0BFFC36A3D3E9002308F0E4FD55
:10A4A00008F0CAFE2D210246504606F0B5F839469E
:10A4B000304608F0B9FF08F059FC2BA3D3E900237C
:10A4C00008F0A8FC2AA3D3E9002308F0CDFD08F08A
:10A4D000B3FE2E210246504606F09EF8DDE900014B
:10A4E00008F0A2FF08F042FC1FA3D3E9002308F004
:10A4F00091FC1FA3D3E9002308F0B6FD08F09CFEF1
:10A500002F210246504606F087F82946204608F0DB
:10A510008BFF08F02BFC14A3D3E9002308F07AFC8E
:10A5200013A3D3E9002308F09FFD08F085FE02463F
:10A530003021504603B0BDE8F04F06F06DB804225C
:10A54000002106F0DDF842462D21504606F064F861
:10A5500032462E21504606F05FF8009A2F215046D1
:10A5600006F05AF82246E3E720FCFFFFFFFF3F43D7
:10A5700000C84E676DC16B44300400202DE9F84FD0
:10A58000614B624F624D00241C60624BC7F8C440AF
:10A590001C60614B87F8CC401C6007F1DC0A07F5B2
:10A5A00080795FFA84F82421404606F05BF85B4B23
:10A5B000297E4AF824000022E254594A4FEA840BCB
:10A5C00002F14000002977D1564949F8241042F899
:10A5D000241040F82410544EAA6A4BF8062006F1C5
:10A5E0000C02E96A4BF8021006F11802296B4BF8CD
:10A5F000021006F12402696B4BF8021006F13002DA
:10A60000A96B4BF802104046252106F02BF806F105
:10A610003C02262142F80B00404606F023F806F1E2
:10A620004802272142F80B00404606F01BF806F1CD
:10A630005402E96B42F80B0006F1600295F84F30C6
:10A640004BF8021006F16C02296C4BF8021006F16F
:10A650007802696C4BF802108436AA6C4BF806201D
:10A6600013B9012385F84F304046FFF703FE01344C
:10A670004046FFF7D5FE032C05F1800591D12B4A0A
:10A6800000231946904642F823100133B3F5807F2A
:10A69000F9D1274CA37ECBB1264E0C25002405F220
:10A6A0008C6761193819042231440434FEF7EAFB3F
:10A6B0000C2CF6D10C35F1E71F4949F824101F493D
:10A6C00042F824101E4A40F8242084E7E37E4BB170
:10A6D000637DB3B1FEF784FA98B1012387F8C030E7
:10A6E000BDE8F88F4FF4FF6540F6D806A5F5FF6189
:10A6F0002846042241440435FEF7C4FBB542F5D197
:10A70000E6E70023EAE700BFE808002078F6FF1F2D
:10A71000300400200409002070070020E703002017
:10A7200048F7FF1FDF09010094F7FF1F0809002009
:10A730000C80FF1F74070020CF090100D70901001A
:10A74000D3090100F7B5014C637801E068070020E8
:10A75000FF2B00F2D186DFE813F02C023F026002EB
:10A76000CF066F029002A102C202CF06CF06CF062B
:10A77000CF06D502E702F80203031F032C033903B7
:10A7800052035F03780385039603A303B003BD035D
:10A79000C203C603D803CF06CF06CF06E503F303F3
:10A7A0000104CF06CF06CF06CF06CF06CF06CF06D1
:10A7B000CF06CF06CF06CF06CF06CF06CF060F04B3
:10A7C000CF06CF06CF06CF06CF06CF06CF06CF06E1
:10A7D000CF06CF06CF06CF06CF06CF06CF06CF06D1
:10A7E000CF06CF06CF06CF06CF06CF06CF06CF06C1
:10A7F000CF06CF06CF06CF06CF06CF06CF06CF06B1
:10A80000CF06CF06CF06CF06CF06CF06CF06CF06A0
:10A81000CF06CF06CF06CF06CF06CF06CF06CF0690
:10A82000CF06CF06CF06CF06CF06CF06CF06CF0680
:10A83000CF061E0427043104440457046104720443
:10A8400085048F049F04B104C104CB04D504CF0652
:10A85000CF06DF04E904F30402050E051205CF0656
:10A86000CF06CF06CF066C05CF0676058405960584
:10A87000CF06A105CF06CF06CF06CF06CF06CF065F
:10A88000CF06CF06CF06CF06CF06CF06CF06CF0620
:10A89000CF06CF06CF06CF06CF06CF06CF060001E4
:10A8A000090112011B012F0143014C0155015E01F9
:10A8B0006701700179018201CF06CF068B01CF06B7
:10A8C0009401CF069D01AF01CF06CA01D301DC017F
:10A8D000F2010802CF06CF0611021A02B305BC0529
:10A8E000CA05CF06CF06CF06CF06D905E805FB057A
:10A8F000CF062302CF06CF06CF06CF062F0654067B
:10A90000CF0672067C068506CF06CF06CF06CF0699
:10A91000CF06CF06CF06CF06CF06CF06CF06CF068F
:10A92000CF06CF06CF06CF06CF06CF06CF06CF067F
:10A93000CF06CF06CF06CF06CF06CF06CF06CF066F
:10A94000CF06CF06CF06CF06CF06CF069106CF069D
:10A950009A06CF06CF06CF06A706D4F80310A07834
:10A96000C9B203B0BDE8F04005F026BBD4F803102F
:10A97000A078C9B203B0BDE8F04005F089BBD4F8B7
:10A980000310A078C9B203B0BDE8F04005F0A4BB45
:10A99000A07805F036FCD4F80310A378C9B228B922
:10A9A000184603B0BDE8F04005F0D4BB184603B02C
:10A9B000BDE8F04005F0A2BBA07805F022FCD4F879
:10A9C0000310A378C9B228B9184603B0BDE8F04017
:10A9D00005F0E0BA184603B0BDE8F04005F0A8BBAA
:10A9E000D4F80310A078C9B203B0BDE8F04005F078
:10A9F000B7BAD4F80310A078C9B203B0BDE8F040EC
:10AA000005F087BCD4F80310A078C9B203B0BDE844
:10AA1000F04005F039BCD4F80310A078C9B203B0F7
:10AA2000BDE8F04005F042BCD4F80310A078C9B2EC
:10AA300003B0BDE8F04005F015BCD4F80310A078D1
:10AA4000C9B203B0BDE8F04005F042BCD4F8031031
:10AA5000A078C9B203B0BDE8F04005F06CBCD4F8F2
:10AA60000310A078C9B203B0BDE8F04005F041BCC6
:10AA7000D4F80310A078C9B203B0BDE8F04005F0E7
:10AA8000D1BAD4F80310A078C9B203B0BDE8F04041
:10AA900005F062BBD4F803000028C0F20A85A47850
:10AAA000B54A02EB8402D2F800319847B34B03EB6E
:10AAB000C413186103B0F0BDD4F803000028C0F23D
:10AAC000F884A278AD4B03EBC2131B7E012B01D09F
:10AAD00005F081FF0028D2BFA94AAA4A92FBF0F2F2
:10AAE0001421A07803B0BDE8F04005F0AFB9D4F868
:10AAF0000310A078C9B203B0BDE8F04005F0DABA9F
:10AB0000D4F80310A078C9B203B0BDE8F04005F056
:10AB100065BAD4F803000028C0F2CB84A278974B22
:10AB200003EBC2131B7E012B01D005F054FF00285C
:10AB3000CABF944A924A92FBF0F21321D1E7D4F8AB
:10AB40000310A078C9B205F085FC0021A07805F0BB
:10AB5000C3F9D4F803100246A07819B142F00402F8
:10AB60000021BFE722F00402BCE7D4F80310A0786C
:10AB7000C9B203B0BDE8F04005F07CBCD4F80310C6
:10AB8000A078C9B203B0BDE8F04005F051BCD4F8DC
:10AB90000310A078C9B203B0BDE8F04005F036BCA0
:10ABA000D4F80310A078C9B203B0BDE8F04005F0B6
:10ABB00009BCA078744A60234343D35CD4F80320D3
:10ABC0002BB9372103B0BDE8F04005F025BD6F4B30
:10ABD00053F820301A44F4E7A5786B4A60236B439E
:10ABE000D35C23B9D4F8032021212846EAE72121A8
:10ABF000284605F037FDD4F80330C01A634B43F8FC
:10AC00002500A5785021284605F02CFDD4F8033006
:10AC1000C01A5F4B43F825004CE7A5785D4BD4F88C
:10AC2000030001225A55544B03EB8503D3F800313E
:10AC3000984724210246D8E7A6784F4DD4F8030060
:10AC400005EB8606D6F8003198470028B8BF404289
:10AC5000C6F8DC002021A07805F004FD43077FF54D
:10AC600029AFA678D4F8030005EB8605D5F80031A6
:10AC70009847242102463046A4E7A0783F4BD4F8F9
:10AC8000032003EBC0139A623B4B03EB8003C3F832
:10AC90001C2103B0BDE8F040FFF7ECBAA5783749B6
:10ACA000394AE07860236B4301EBC511D35C4872ED
:10ACB00043B98A7A897D8DE803000621284605F08C
:10ACC00081FCF7E61021284605F006F9E37820F428
:10ACD000F852DB0842EA03221021284602E7A07856
:10ACE000E2782649284C6023434301EBC011E35C22
:10ACF0008A72002B7FF4DEAE8C7D0194497A00913C
:10AD00000621DCE70121A07805F0ACFCD4F8033083
:10AD100020F00A02DF0748BF42F002029E0701D579
:10AD200042F008020121D8E00121A07805F09AFC48
:10AD3000D4F8033020F00502DD0748BF42F00102DD
:10AD40009807EFD542F00402ECE7D4F80320012A7B
:10AD500000F2AF83A178094B03EBC113DA75A9E6C2
:10AD6000A578054BD4F8030003EB8503D3F8003135
:10AD700098472521024638E778F6FF1F3004002067
:10AD8000B50010000024F400B4050020D403002016
:10AD9000EC030020E7030020A078BC4BD4F803208C
:10ADA00003EBC0131A63BA4B03EB8003C3F83421DF
:10ADB0006FE7A078B54BD4F8032003EBC013DA6239
:10ADC000B34B03EB8003C3F8282162E7A678B04DAC
:10ADD000D4F8030005EB8603D3F800319847272108
:10ADE0000246304605F018FCA378D4F8030005EBC2
:10ADF0008305D5F800319847C5F870015AE6A07868
:10AE0000A24BD4F8032003EBC0135A63A04B03EB0F
:10AE10008003C3F840213CE7A6789D4DD4F8030099
:10AE200005EB8603D3F800319847262102463046C9
:10AE300005F0F2FBA378D4F8030005EB8305D5F801
:10AE400000319847C5F8640134E6A0788F4BD4F8F8
:10AE5000032003EBC0139A638D4B03EB8003C3F80D
:10AE60004C2116E7A078894BD4F8032003EBC013DC
:10AE7000DA63874B03EB8003C3F87C2103B0BDE8A2
:10AE8000F040FFF7CDBAA078804BD4F8032003EB55
:10AE9000C0131A647E4B03EB8003C3F88821EDE7EF
:10AEA000A0787A4BD4F8032003EBC0135A64784B94
:10AEB00003EB8003C3F89421E0E7A078734BD4F848
:10AEC000032003EBC0139A64714B03EB8003C3F8B8
:10AED000A021D3E7D4F803203321A07872E6D4F878
:10AEE00003203421F9E70121A07805F0BBFBD4F859
:10AEF000033020F0C002D90748BF42F040029B0750
:10AF00007FF510AF42F080020CE70121A07805F038
:10AF1000A9FBD4F803301B0220F4407203F4407301
:10AF20001A43FFE60121A07805F09CFBD4F803301A
:10AF300020F01002002B3FF4F5AE42F01002F1E6D3
:10AF40000121A07805F08EFBD4F8033020F0200218
:10AF5000002B3FF4E7AE42F02002E3E6D4F80330E2
:10AF6000013BFE2B00F2A582A078484BE27803EB70
:10AF7000C01383F84F2081E7A078464A60234343FB
:10AF8000D35C002B3FF496ADD4F8031003B0BDE8BA
:10AF9000F04003F0BBB9A0783E4BD4F80320602109
:10AFA00001FB00335A600DE63A49A078D4F803203B
:10AFB000602303FB001361219A6003E6A078354A01
:10AFC000602303FB0023D4F803201A731C2105F02F
:10AFD00049FBD4F80320C0F3080040EA02421C21D8
:10AFE0007BE7A0782B4A602303FB0023D4F80320DF
:10AFF000DA811C2105F036FBD4F8033000F47F021F
:10B00000C3F308031A43EAE72249A078D4F80320DF
:10B01000602303FB001359211A61D3E5A078D4F80B
:10B0200003201C4C60234343E118E35CD2B20A7551
:10B03000002B3FF43FAD8B7D01924A7D0FE0A0785D
:10B04000D4F80320134C60234343E118E35CD2B2ED
:10B050004A75002B3FF42EAD8B7D097D0191009246
:10B0600000224DE60B49A078D4F80320602303FBAF
:10B0700000135A211A62A5E50649A078D4F80320E6
:10B08000602303FB00135B215A629BE53004002020
:10B0900078F6FF1FB4050020A078A849D4F8032053
:10B0A000602303FB0013D1B29A62C2F3072293F824
:10B0B0002C300191009200225D2100E6A0789F498A
:10B0C000D4F80330602202FB0012D362926AD1B23C
:10B0D000C2F3072201910092DBB2ECE79749A07816
:10B0E000D4F80320602303FB00135E211A6369E593
:10B0F0009249A078D4F80320602303FB00131821A1
:10B100009A615FE58D49A078D4F80320602303FBA2
:10B1100000131921DA6155E58849A078D4F8032095
:10B12000602303FB00135C215A634BE58349A0783D
:10B13000D4F80320602303FB00135F219A6341E5E9
:10B14000A078D4F803307D4C60224243A118A25C61
:10B15000DBB28B75002A3FF4ADAC0A7D6CE7D4F806
:10B160000330022B00F2A581A278754B1344E278DC
:10B1700083F8E8209EE4D4F803202021ADE6D4F83B
:10B180000330032B00F29581DFE803F002172A4118
:10B19000A0786A4D602707FB00F3EE5C16B1002231
:10B1A000EA5487E44FF44002072105F0A9FAA37896
:10B1B00007FB035383F849607CE4A0784FF4400216
:10B1C000072105F09DFAA0785C4A60234343D1181B
:10B1D000002481F849405B4C01212154D15469E499
:10B1E000A078564D602606FB00F3EB5C5BB94FF48C
:10B1F0004002072105F076FAA37806FB03530122EB
:10B2000083F8492056E406224F4B1A7052E4A07886
:10B210004A4D602606FB00F3EB5C002BF3D14FF4A4
:10B220004002072105F06CFA4FF400020721A078D4
:10B23000E0E74249A078D4F80320602303FB001321
:10B240005221DA63BEE43D4AA078E178602303FB33
:10B2500000235A6C83F84010019193F84130009319
:10B260000CE0A078354AE178602303FB002383F8E3
:10B2700041105A6C93F840308DE80A00D3B2632134
:10B28000C2F307221BE52D49A078D4F803206023E0
:10B2900003FB00135A6493F84010DDE7D4F8033041
:10B2A000082B00F206810A21A07805F0DBF9D4F81A
:10B2B000033020F00F02C3F108031A430A210CE601
:10B2C000A278224B03EBC213D4F803201A72FFF7C3
:10B2D000F1BBA5781A4BD4F8030003EB8503ED010D
:10B2E000D3F800319847194B5851FFF7E3BBA578C5
:10B2F000134AD4F8030002EB8502D2F800319847D4
:10B30000124B03EBC5135860FFF7D4BBA0780F496D
:10B310000A4AE4786023434301EBC011D35C8C7587
:10B32000002B7FF4C7AB8A7AE7E4D4F80310A07847
:10B3300003B0BDE8F04004F0AFBC00BFB40500208E
:10B3400078F6FF1FE7030020FC08002030040020EF
:10B35000A0786A4DD4F8032005EBC011B1F84C3049
:10B360009A423FF4A7AB60234343654EF35C002B46
:10B370007FF449AF0C23A1F84C20009392B2042330
:10B380000A2105F0CBF9A07805EBC0135421DA6946
:10B39000002AB8BF524205F03FF9A07805EBC0156E
:10B3A000EB69002B4FF000524FF0070177DA03B042
:10B3B000BDE8F04005F096B9A578514A514E60239A
:10B3C0006B43D75C97B15021284605F04BF9D4F870
:10B3D0000330C01A46F82500A5782121284605F03B
:10B3E00041F9D4F80330C01A474B13E4D4F80320D2
:10B3F0005021284605F010F9A37846F82370FFF78E
:10B4000059BBA0783D4DD4F8032005EBC013DB6990
:10B410009A423FF44FAB602343433949CB5C002B46
:10B420007FF4F1AE002AB8BF5242542105F0F4F87F
:10B43000A078D4F8033005EBC015EB61B1E7A07834
:10B440002E4BD4F8032003EBC01353211A62FFF7ED
:10B45000B9BBA278294B03EBC213D4F803205A627C
:10B46000FFF728BBA078254BD4F8032003EBC013CB
:10B4700015219A82254B5A43FFF7A4BBA2781F4B94
:10B4800003EBC213E27883F84E20FFF713BBD4F826
:10B490000310A0784FF0805209B1002187E703B074
:10B4A000BDE8F04005F02CB9D4F803201AB1012A08
:10B4B00012D00422A8E6A0781049154B01EBC01168
:10B4C00003EB80030A76134AC3F80021C3F8D020A7
:10B4D000C3F81021FFF7EEBAA07808490C4B01EB36
:10B4E000C01103EB80030A760B4AC3F800210B4A14
:10B4F000C3F8D0200A4AEBE7032285E63004002097
:10B50000B4050020EC030020D403002000710200E9
:10B5100078F6FF1FDF090100CF090100D7090100FC
:10B52000D3090100F8B5214C2718064697F8AC312D
:10B53000002B39D004EB80042521D4F858211C4D70
:10B5400005F06AF8D4F870212721304605EBC615BE
:10B5500005F062F8D4F864212621304605F05CF845
:10B56000D4F81C31AB62D4F82831EB62D4F8343112
:10B570002B63D4F840316B63D4F84C31AB63304665
:10B58000FEF778FED4F87C31EB63D4F888312B6475
:10B59000D4F894316B64D4F8A031AB643046FEF734
:10B5A0003FFF002387F8AC31F8BD00BF78F6FF1FDE
:10B5B000300400202DE9F04FBC4C2DED028BA0781B
:10B5C000022887B002D96378022B06D16378012B59
:10B5D0006ED007D3022B00F0E48007B0BDEC028BE5
:10B5E000BDE8F08FB24FDFF8D8A2DFF8E8B2DFF89D
:10B5F000D4820025B946A378AB4209D009EBC31326
:10B6000093F84E30002B46D097F84E209A4242D104
:10B61000EEB2304602F0A8FE002305F80A3005F825
:10B620000B304FF000620121304605F05BF8FB7DE6
:10B63000BBBB05222021304604F0EEFF15F8083090
:10B640004BB19C4B242153F82520304604F0E4FFF5
:10B65000002305F808303046FFF764FF4FF08052B2
:10B660000721304605F04CF84FF0006207213046C4
:10B6700005F038F86023904A6B439B5CD4F80320B4
:10B680008BB93721304604F0C7FF4FF0006201212B
:10B69000304605F035F80135032D07F18007AAD1B2
:10B6A0009BE70622C6E7854B53F825301A44E8E7A6
:10B6B000DFF8FC81DFF81CA2DFF81CB20026C146CF
:10B6C000A378B34209D009EBC31393F84E30002B93
:10B6D00054D098F84E209A4250D1F5B2284602F044
:10B6E00043FE774A0023B35406F80A304FF0006255
:10B6F0000121284604F0F6FF98F817306BB90522AF
:10B700002021284604F088FF16F80B30012B3BD08F
:10B7100005D3022B3AD0002708E00622F0E73721B4
:10B72000284604F09FFFD4F803700744654BF25C91
:10B7300052B1604A019352F826202421284604F091
:10B740006BFF019B0022F2542846FFF7EBFE4FF0FF
:10B7500080520721284604F0D3FF4FF000620721F2
:10B76000284604F0BFFF3A463721284604F054FF2C
:10B770004FF000620121284604F0C2FF0136032E7B
:10B7800008F180089CD128E72121C9E750212846EB
:10B7900004F068FF4C4B53F82670C71BD4F8030025
:10B7A000C3E7D4F80390B9F11E0F00F3848210F0C0
:10B7B000400500F0B78100231946012540FA03F245
:10B7C00012F0010215BF02AA02AED554F25403F1E1
:10B7D000010318BF0131032BF0D101297EDC9DF854
:10B7E0000830002B5ED19DF80930002B5CD19DF80C
:10B7F0000A308BB10225334F7B5D53B1334B03EBE2
:10B8000085032421D3F8DC20284604F005FF00231B
:10B810007B552846FFF786FE294FDFF8B880DFF812
:10B8200090900025A3782B41D90737D5EEB230464A
:10B8300002F09AFD0023EB5505F8083009EBC5131B
:10B84000DB7D002B40F0608105222021304604F092
:10B85000E3FE4FF080520721304604F051FF4FF0D5
:10B8600000620721304604F03DFF6023124A6B431B
:10B870009B5C174A002B40F04981D4F8033003EB5E
:10B8800043032B4452F823203721304604F0C4FEF2
:10B890004FF000620121304604F032FF0135032DE4
:10B8A000C0D19AE60025A6E70125A4E76807002095
:10B8B0003004002054F7FF1FB4050020D4030020FB
:10B8C00028040020E7030020EC03002078F6FF1F87
:10B8D00074070020E403002060F7FF1FC34BC44E31
:10B8E000DFF820830C2202FB093900256027A378AA
:10B8F0007B43E8B2F35C0DF10C0B2121002B40F0EF
:10B90000FD8004F0AFFE59F82530C31A83EAE370D6
:10B91000A0EBE3704BF825000135032DE7D10023A0
:10B920001F464FF0FF3202A9D8B2C95C29B15BF8BB
:10B9300023109142C4BF07460A460133032BF2D1BC
:10B94000AC4BDA5D9A465AB1AB4B03EB870324212B
:10B95000D3F8DC20384604F05FFE00230AF80730F5
:10B960003846A54EA54DFFF7DDFDBB004FF00008A2
:10B970001E4402AA5FFA88F912F80820002A00F093
:10B98000B4804F4500F0B1805BF82820019307EEAA
:10B99000902A06AA1A44B8EEE77A52ED037AF8EE36
:10B9A000E77A242187EE278A4846D6ED377AF8EEE3
:10B9B000E77A67EE887AFDEEE77A17EE902A04F0D0
:10B9C0002BFED6ED567AF8EE677A252167EE887A57
:10B9D0004846FDEEE77A17EE902A04F01DFED6EDFC
:10B9E0005C7AF8EE677A272167EE887A4846FDEEA2
:10B9F000E77A17EE902A04F00FFED6ED597AF8EEAA
:10BA0000677A262167EE887A4846FDEEE77A17EED8
:10BA1000902A04F001FE794B03EBC712D2ED0A7AAB
:10BA2000F8EE677A484667EE887AFDEEE77AC5ED6C
:10BA30000A7AD2ED0B7AF8EE677A67EE887AFDEE35
:10BA4000E77AC5ED0B7AD2ED0C7AF8EE677A67EEFD
:10BA5000887AFDEEE77AC5ED0C7AD2ED0D7AF8EE34
:10BA6000677A67EE887AFDEEE77AC5ED0D7AD2ED5A
:10BA70000E7AF8EE677A67EE887AFDEEE77AC5ED22
:10BA80000E7AFEF7F7FBD6ED5F7AF8EE677A484656
:10BA900067EE887AFDEEE77AC5ED0F7AD6ED627A29
:10BAA000F8EE677A67EE887AFDEEE77AC5ED107AF0
:10BAB000D6ED657AF8EE677A67EE887AFDEEE77A7A
:10BAC000C5ED117AD6ED687AF8EE677A27EE888AA6
:10BAD000BDEEC88A85ED128AFEF7A2FC4849019B9B
:10BAE00001220AF8082008F8012008F10108B8F13D
:10BAF000030F05F180057FF43CAF8DE604F0B2FD45
:10BB000058F82530C01AFEE606229EE6D4F8033027
:10BB100003EB43032B4452F823203A4B53F82530D0
:10BB20001A44B1E6020675D5374FDFF8E480DFF836
:10BB3000CC90A3782B41DB0746D5EEB2304602F01D
:10BB400013FC0023EB5505F8083009EBC513DB7D2A
:10BB5000002B3DD10522DFF89CA02021304604F0C7
:10BB60005BFD15F80A304BB1284B242153F82520F2
:10BB7000304604F051FD002305F80A303046FFF747
:10BB8000D1FC4FF080520721304604F0B9FD4FF050
:10BB900000620721304604F0A5FD6023144A6B4380
:10BBA0009B5C124AB3B9D4F8033003EB43032B4434
:10BBB00052F823203721304604F02EFD4FF000626A
:10BBC0000121304604F09CFD0135032DB1D104E57F
:10BBD0000622C0E7D4F8033003EB43032B4452F8AA
:10BBE0002320084B53F825301A44E3E7740700205C
:10BBF000B4050020E703002078F6FF1F3004002082
:10BC000024F8FF1FD40300202804002054F7FF1F4E
:10BC1000E403002002284ED802F0A6FBA078284BAF
:10BC20001D54284B1D54284B03EBC013DB7D002B08
:10BC30003AD10522202104F0EFFC244DA0782B5CA2
:10BC400053B1234B03EB80032421D3F8DC2004F011
:10BC5000E3FCA3780022EA544FF080520721A07839
:10BC600004F04EFD4FF000620721A07804F03AFD89
:10BC7000A078184A60234343D15CD4F80330164AB5
:10BC800003EB4303034452F8232079B9372104F02E
:10BC9000C3FCA0784FF00062012107B0BDEC028B1D
:10BCA000BDE8F04F04F02CBD0622C3E70B4B53F860
:10BCB00020301A44EAE70A4B04221A708DE400BFD0
:10BCC00028040020E403002030040020E7030020C3
:10BCD00078F6FF1FB405002074070020D40300206D
:10BCE000FC0800202DE9F341C44FC5493A784A7059
:10BCF00064230B70292AD7F803304B603C460D466D
:10BD000001F0648000F2EA80142A00F046845DD8D5
:10BD10000A2A00F0E78122D8052A00F0D78111D83D
:10BD2000022A00F0C78105D8012A00F0BE81022353
:10BD30002B70BCE1032A00F0C081042AF7D1FFF781
:10BD400039FCB4E1072A00F0C781C0F0C281082A9B
:10BD500000F0C581092AEAD1FDF790FFA7E10F2A7B
:10BD600000F0958317D80C2A00F04683C0F02F838B
:10BD70000D2A00F053830E2AD9D1BA78022A40F056
:10BD8000838378781F2800F27483002B40F06E8341
:10BD9000FCF73CFE8BE1112A01F02683C1F01D83E4
:10BDA000122A01F02883132AC1D17978954A0929EA
:10BDB00000F2C983DFE811F0C403CF03D203D50337
:10BDC000D903E003E303E603E903DE031F2A00F0DF
:10BDD000E8854DD8192A00F0A58419D8162A00F054
:10BDE0008B84C0F0F983172A00F08A84182A9ED128
:10BDF000854AD2F8C830002B00F05981013BC2F8C7
:10BE0000C83002EB8303D3F8B031C2F8C4304EE13E
:10BE10001B2A00F0A384C0F093841C2A00F09085B4
:10BE20001E2A84D17A781E2A00F2E082BE78022E81
:10BE300000F28C8502EB42007449304441F8203016
:10BE4000734B9B7E002B00F03281002A00F02F8183
:10BE5000032313FB02630C20013A424302F5D36033
:10BE6000042201EB830102FB0600FCF7CAFF1EE17E
:10BE7000242A00F0A58611D8212A00F03486C0F0CB
:10BE8000DE85222A00F08586232A7FF450AF5D4BA1
:10BE90001B68C7F80330FDF7F1FE08E1262A00F021
:10BEA000CC86C0F0C086272A00F0EF86282A7FF4CF
:10BEB0003EAFFF2B00F3FB807A780B2A00F28287DB
:10BEC000DFE812F0F50600070B0716072207300718
:10BED0003B07460751075A0762076E07432A01F0DE
:10BEE000C58369D8332A01F0578232D82E2A01F04F
:10BEF00025821CD82B2A01F08F80C1F006802C2AC5
:10BF000001F018812D2A7FF412AF7A780B2A01F202
:10BF10001182DFE812F0AE09B709C009C909D309D7
:10BF2000DF09E809F109FA09030A0F0A090A302AA8
:10BF300001F01782C1F00A82312A01F01E82322AF2
:10BF40007FF4F5AE2F4B1B68C7F80330FEF7E4F81B
:10BF5000ADE0382A01F05A8213D8352A01F02D823B
:10BF6000C1F02082362A01F03382372A7FF4DFAE17
:10BF7000284A1268FF2A00F29A80274941F82230A5
:10BF800095E0402A01F06A830DD8392A7FF4CFAEBC
:10BF9000204B1B68FF2B00F28A801A4A11681E4A48
:10BFA00042F8231083E0412A01F05C83422A7FF4A7
:10BFB000BEAE02F09DF97AE0842A01F0868336D87D
:10BFC000502A01F047820DD8452A01F05783C1F06D
:10BFD0005183462A01F05683472A7FF4A8AE02F027
:10BFE0008CF964E0812A01F0518317D8802A7FF40C
:10BFF0009EAE054B002283F8C02058E06807002061
:10C00000FC080020E808002078F6FF1F74070020D5
:10C010000C80FF1F0409002008090020822A01F07B
:10C020004E83832A7FF483AEFDF764F83FE0892ACC
:10C0300001F0088416D8862A01F06183C1F0598383
:10C04000872A01F0D183882A7FF471AE7B78012B97
:10C0500001F0AF83C1F09A83022B01F0B383032375
:10C060000B7024E08D2A01F03E840FD88A2A01F05B
:10C0700002848C2A7FF45BAE7E78002E01F014845B
:10C08000012E01F0218403230B7010E0F22A01F04D
:10C090007984FF2A7FF44BAE40F2D242934206D11C
:10C0A000AF4B012283F82C2201E0FDF7C9FF02B05B
:10C0B000BDE8F081FEF730F8F9E7BB78022B02D833
:10C0C000FEF798F8F3E704232B70F0E7FEF73AFB4E
:10C0D000EDE7FDF739F8EAE7FCF7FEFFE7E7FCF7E5
:10C0E000FBFFE4E7BB78022B00F0BD80032B00F0E0
:10C0F000BF80002B40F064817B78502B00F0828061
:10C1000028D8462B6FD010D8422B66D006D8402BAB
:10C1100049D0412B5DD003232B7049E0442B5FD0E5
:10C12000452BF8D18F4B5B7955E04B2B61D009D86B
:10C13000472B5BD0492BEED18A4BDB7D003318BFF8
:10C14000012348E04D2B5AD056D34F2BE3D1854BDA
:10C150005B7E40E0802B64D012D8532B58D006D899
:10C16000512B52D0522BD6D17E4B1B6A33E0552B2C
:10C1700054D050D3562BCED17A4B93F824302AE0AA
:10C18000832B5CD007D8812B4FD0822BC3D1744B2B
:10C19000D3F8C4301FE0852B58D054D3FF2BBAD12D
:10C1A000714B1B78CAE745F2FF70FCF751FE6860DF
:10C1B0006E4B1B78002B3FF47AAF6D4B6A681A60A8
:10C1C0006C4B002A40F0FE801A6842F008021A60A8
:10C1D0006DE7644B1B786B60EAE7624B5B78FAE7CC
:10C1E000604BDB69F7E75F4BDB68F4E75D4B9B680F
:10C1F000F1E75C4BDB78EEE75A4B9B78EBE7594B6A
:10C200005B7DE8E7574B9B7DE5E7564B1B7DE2E7FF
:10C21000544B1B69DFE7534B9B7EDCE7514BDB7EC6
:10C22000D9E74F4B93F8C030D5E74D4B93F8C0306A
:10C23000A3F1040CDCF1000343EB0C03CBE7484B08
:10C24000D3F8EC30C7E74C4B1B68C4E7444A4B4873
:10C25000D2F8F03043F2390100FB0313C2F8F0309A
:10C2600023F00043B7E77A78454B53F82230B2E722
:10C270007B782E2B3FF64FAF01A252F823F000BF80
:10C280003DC3000041C3000047C3000017C10000C8
:10C2900017C1000017C1000017C1000017C100003E
:10C2A00017C10000B1C10000B1C10000B1C1000060
:10C2B00017C1000017C1000017C1000017C100001E
:10C2C00017C1000017C1000017C1000017C100000E
:10C2D00017C1000017C1000017C1000017C10000FE
:10C2E00017C1000017C1000017C100004BC30000B8
:10C2F00051C3000055C3000059C3000089C30000AA
:10C300008DC3000017C1000017C1000017C1000055
:10C3100017C1000017C1000017C1000093C300003F
:10C3200097C300009DC30000A3C30000A9C3000081
:10C33000AFC30000B5C30000BBC30000114B83E7CF
:10C34000104B5B6847E70F4B51E70E4B1B7E42E7F4
:10C350000C4B64E70B4BFBE60A4B1B7F3BE700BF34
:10C3600078F6FF1F0C80FF1FF6080020F70800205A
:10C37000E808002070070020F80800206D4EC64134
:10C3800008090020E00600209A4B45E7994B5B7FA7
:10C3900021E7984BE9E6974B5B6A1CE7954B9B6A54
:10C3A00019E7944BDB6A16E7924B1B6B13E7914B33
:10C3B0005B6B10E78F4B9B6B0DE78E4BDB6B0AE7DC
:10C3C0000423A9E61A6822F008021A606FE6BB7817
:10C3D000022B0ED17878372808D800F5FF708649EF
:10C3E000800004220144FCF70CFD60E603232B705F
:10C3F0005DE604230B705AE6BB78022B0BD17878EC
:10C400003728F3D800F5FF707B49800004220144EF
:10C41000FCF738FD4BE604230B7048E6B878022899
:10C420003FF651AE7B78012B08D004D3022B08D005
:10C4300003230B703BE603F055F838E603F05AF897
:10C4400035E603F05FF86D4B68601B78002B3FF416
:10C450002EAE6B4B18606B4B1A6818B942F008028D
:10C460001A6024E622F008021A6020E6FCF7BAFA05
:10C470001DE6FF287FF41BAE5F1C0ABF604B184609
:10C480001868FCF7D7FA12E604230B700FE6BE78A3
:10C49000012E29D004D3022E49D004230B700FE0C3
:10C4A0007878092803D8FCF7D7FA686008E00A28EA
:10C4B00015D1554B1B6983F40073C3F340234B60C4
:10C4C0004E4B1B78002B3FF4F2AD4D4B6A681A605F
:10C4D0004C4B82BB1A6842F008021A60E7E5FF285D
:10C4E000EED1FCF7F1FAE0E77878092802D003F002
:10C4F0000DF9DAE70020FCF7FFFA04463046FCF7B6
:10C50000FBFA06460220FCF7F7FA8642D4BF002366
:10C5100001239C4209DD331C18BF01231BB986424D
:10C520003446B8BF04466C60CAE7031CF4E7787869
:10C53000FCF7ABFAB9E71A6822F008021A60B6E510
:10C5400010681844106012682E4B0ABB1A6842F03B
:10C5500008021A60ABE51068C01AF3E71068584388
:10C56000F0E7106890FBF3F0ECE7116891FBF3F053
:10C5700003FB10131360E6E710681840E2E7106849
:10C580001843DFE710685840DCE71368DB43F1E746
:10C590001A6822F008021A6089E5194A1168194AD6
:10C5A0008B4213680ADA23F0030343F00403136099
:10C5B000136869B943F00803136078E50BBF23F0F3
:10C5C000060323F0050343F0010343F00203EEE703
:10C5D00023F0080313606AE57A780C2A3FF667AD0A
:10C5E000DFE802F0141D262F38414B545D666F784A
:10C5F000810000BFE006002010010020F7080020A5
:10C60000E80800207007002080F00F40B04A126850
:10C6100016077FF54CADAF4AC2F8C43047E5AC4AC7
:10C62000126815073FF543ADAA4AC2F8C4303EE58B
:10C63000A74A1268D4077FF53AADA64AC2F8C430BB
:10C6400035E5A34A1268D0073FF531ADA14AC2F8DB
:10C65000C4302CE59E4A126851077FF528AD9D4AEB
:10C66000C2F8C43023E59A4A126812F0050F3FF46D
:10C670001EAD984AC2F8C43019E5954A126892076F
:10C680007FF515AD934AC2F8C43010E5904A1268A0
:10C6900097073FF40CAD8F4AC2F8C43007E58C4AC7
:10C6A0001268D6067FF503AD8A4AC2F8C430FEE4AC
:10C6B000874A126895067FF5FAAC864AC2F8C430FC
:10C6C000F5E4834A126854067FF5F1AC814AC2F85A
:10C6D000C430ECE47E4A126810067FF5E8AC7D4A6F
:10C6E000C2F8C430E3E47A4A1268D1057FF5DFACC2
:10C6F000784AC2F8C430DAE4764AC2F8C430D6E4E4
:10C70000744AD2F8C81007293FF6D1AC481C02EB96
:10C710008101C2F8C800D2F8C400C1F8B001C2F863
:10C72000C430C4E47B782E2B03D86B4A0121D1544A
:10C73000BDE4FF2B7FF45AAE664B01221A70B6E4BB
:10C740007B782E2B03D8644A0021D154AFE4FF2B11
:10C750007FF44CAE5F4B00221A70A8E45D4D95F853
:10C76000CC2072B95A1C04BF5C4B1B680A2058438A
:10C77000C5F8D001FBF782FF0123C5F8D40185F885
:10C78000CC306378042B3FF692ACDFE803F003442F
:10C7900071A91A00FBF772FFD5F8D431C01A00282E
:10C7A000D5F8D031B8BF4042984295BFD5F8C430D3
:10C7B000002303F1FF3385F8CC3098BFC5F8C430AF
:10C7C00075E4A07802F09EFE38B9414A85F8CC00A5
:10C7D000136823F01003136069E4D5F8D031A3B1D6
:10C7E000FBF74CFFD5F8D431C01A0028D5F8D0316A
:10C7F000B8BF4042984208D9354A002385F8CC306A
:10C80000136843F01003136051E4D5F8C430013BC2
:10C81000C5F8C4304BE4A0780F2103F023FF10F0DB
:10C82000010408D02A4A002385F8CC30136823F08D
:10C83000100313603BE4D5F8D0319BB1FBF71EFF2A
:10C84000D5F8D431C01A0028D5F8D031B8BF40424D
:10C85000984207D91E4A85F8CC40136843F010036C
:10C86000136024E4D5F8C430013BC5F8C4301EE49D
:10C87000A0780F2103F0F6FE10F0800408D0144ACF
:10C88000002385F8CC30136823F0100313600EE406
:10C89000D5F8D031A3B1FBF7F1FED5F8D431C01AE9
:10C8A0000028D5F8D031B8BF4042984208D9084A8C
:10C8B00085F8CC40136843F010031360FFF7F7BB13
:10C8C000D5F8C430013BC5F8C430FFF7F0BB00BF5A
:10C8D0007007002078F6FF1F31070020E8080020CD
:10C8E000A0780F2103F0BEFE10F4807409D0AD4A89
:10C8F000002385F8CC30136823F010031360FFF792
:10C90000D6BBD5F8D031A3B1FBF7B8FED5F8D431FA
:10C91000C01A0028D5F8D031B8BF4042984208D993
:10C92000A04A85F8CC40136843F010031360FFF76A
:10C93000BEBBD5F8C430013BC5F8C430FFF7B7BB68
:10C94000994B002283F8C020FFF7B1BBFF2E7FF484
:10C95000BAAB964E72B90C25002405F28C672919E2
:10C960003819042231440434FCF74BFA0C2CF6D16C
:10C970000C35F1E700254FF003080C27607818FB11
:10C9800000510138784300F5D36000EB85000422A4
:10C9900006EB81010135FCF734FA032DEED1FFF7E8
:10C9A00086BB7B781E2B3FF621ADBA78022A1BD8B6
:10C9B00003EB430313447D4A52F823207C4B4A6027
:10C9C0001B78002B3FF473AB7A4B1A60754B2AB976
:10C9D0001A6842F008021A60FFF769BB1A6822F071
:10C9E00008021A60FFF763BBFF2A7FF46CAB6F4E3F
:10C9F00073B90C25002405F28C6729193819042213
:10CA000031440434FCF73EFA0C2CF6D10C35F1E736
:10CA100000254FF003080C27607818FB00510138FF
:10CA2000784300F5D36000EB8500042206EB81011A
:10CA30000135FCF727FA032DEED1FFF738BB7E78DE
:10CA40001E2E3FF6D3ACBF783B062CD5574FDFF8F0
:10CA50006C810025A3782B41DE0709D5667821215A
:10CA6000E8B203F0FFFD06EB46062E4447F8260029
:10CA700098F81A3093B16278531ED9B227290DD88D
:10CA80000C200321584311FB025100F5D36004220E
:10CA900007EB810100EB8500FCF7B3F90135032DAD
:10CAA000D8D1FFF704BB022F3FF60DAB212138464A
:10CAB00003F0D8FD06EB46063C4D63783E44032167
:10CAC00045F82600A0785A1E11FB03010C2353439E
:10CAD00003F5D363042205EB810102FB0030FCF770
:10CAE00090F9FFF7E4BA7A78324B0A2A0CD8DFE8DB
:10CAF00002F006151A1F252D32373C4145002E49FC
:10CB00001A6809680A441A601A68264B002A3AD142
:10CB10001A6842F008021A60FFF7C9BA26491A6873
:10CB20000968521AEFE7244A196812684A43EAE78B
:10CB300021491A68096892FBF1F2E4E71E4A186875
:10CB4000116890FBF1F201FB1202DCE71A491A6846
:10CB500009680A40D7E718491A6809680A43D2E702
:10CB600015491A6809684A40CDE713490A68D24353
:10CB70000A60C9E71968104A1160C5E70E4A1968CA
:10CB800010681860F8E71A6822F008021A60FFF7C8
:10CB90008EBA084B1B68C7F80330FDF7D3FDFFF7CB
:10CBA00086BA00BF7007002078F6FF1F74070020C8
:10CBB000F7080020E8080020040900200C80FF1F6F
:10CBC0007B78052B3FF673AADFE803F0030A111800
:10CBD0001F26BB4A136803F00F031360FFF767BA01
:10CBE000B74A136823F010031360FFF760BAB44A22
:10CBF000136823F020031360FFF759BAB04A136893
:10CC000023F040031360FFF752BAAD4A136823F0D4
:10CC100080031360FFF74BBAA94A136823F48073AB
:10CC20001360FFF744BA79782E293FF6DFABA54AA7
:10CC300002EB81025360FFF73ABAA24BA24AD3F843
:10CC4000D8111160A14AD3F8DC111160D3F8E021AA
:10CC5000C3F8C4209A4AD3F8E4111160D3F8E8214C
:10CC600083F8CC20D3F8EC21C3F8D421D3F8F021F9
:10CC7000C3F8D02193F8F411954A505C08B1012013
:10CC8000505400225A70FFF712BABA78022A3FF6BF
:10CC90001AAA7B781E2B3FF6A9AB03EB4303134480
:10CCA000894A11688B4A42F82310FFF700BA8A4A72
:10CCB000B87852F8233052F82010194442F8201066
:10CCC000FFF7F5B9844AB87852F8233052F82010AB
:10CCD000C91A42F82010FFF7EAB97F4AB97852F82A
:10CCE000233052F82100434342F82130FFF7DFB9E7
:10CCF000794AB87852F8233052F8201091FBF3F1BA
:10CD000042F82010FFF7D3B9734AB97852F82300DC
:10CD100052F8214094FBF0F300FB134342F821301A
:10CD2000FFF7C5B96C4AB87852F8233052F8201092
:10CD3000194042F82010FFF7BAB9674AB87852F89C
:10CD4000233052F82010194342F82010FFF7AFB9F2
:10CD5000614AB87852F8233052F82010594042F80E
:10CD60002010FFF7A4B95C4AB97852F82330DB43AE
:10CD700042F82130FFF79BB9574A52F82310BB788D
:10CD800042F82310FFF793B9534AB97852F8234079
:10CD900052F8210042F8214042F82300FFF787B9FA
:10CDA0004D4AB97852F8233052F82110994240F395
:10CDB0004E82434A136823F0030343F004031360D5
:10CDC000FFF775B903232B70FFF771B97B780B2B35
:10CDD00000F29780DFE803F006111C2733414C571F
:10CDE000626B828DB9783C4A374852F8213000682E
:10CDF000034442F82130FFF75AB9B978364A32482D
:10CE000052F8213000681B1A42F82130FFF74FB961
:10CE1000B978314A2C4B52F821001B68434342F841
:10CE20002130FFF744B9B9782B4A274852F821300E
:10CE3000006893FBF0F342F82130FFF738B9B97876
:10CE4000254A214B52F82140186894FBF0F300FB6F
:10CE5000134342F82130FFF72AB9B9781E4A1A481D
:10CE600052F821300068034042F82130FFF71FB923
:10CE7000B978194A144852F821300068034342F83F
:10CE80002130FFF714B9B978134A0F4852F821300E
:10CE90000068434042F82130FFF709B90A4BB978DE
:10CEA0001B680D4ADB4342F82130FFF700B9064BFF
:10CEB000BA781968084B43F82210FFF7F8B800BF9A
:10CEC0007007002078F6FF1FE80800200409002002
:10CED000310700207407002008090020B9789B4A18
:10CEE0009B4B52F821001C6842F821401860FFF764
:10CEF000DEB8964BBA7853F82220954B1B689A42BD
:10CF000055E703230B70FFF7D2B87978904B914A1D
:10CF10000B2978D8DFE801F006161D242C363D4495
:10CF20004B51565FB878894951F820101868014470
:10CF300019601B68002B69D1136843F00803136064
:10CF4000FFF7B5B8BC788148196850F82400091A71
:10CF5000EEE77E49B87851F8200019684143E7E7C9
:10CF6000BC787A48196850F8240091FBF0F1DFE7AB
:10CF70007649B8781C6851F8200094FBF0F100FB6A
:10CF80001141D5E7B878714951F82010186801406F
:10CF9000CEE7B8786D4951F8201018680143C7E70B
:10CFA000B8786A4951F8201018684140C0E7B8784D
:10CFB000664951F82010C943BAE7B878634951F877
:10CFC0002010B5E7B87861491D6851F820401C6011
:10CFD00041F82050ADE75D49B87851F82000196854
:10CFE0008842116805DA21F0030141F00401116063
:10CFF0009FE70BBF21F0060121F0050141F001017F
:10D0000041F00201F3E70321297092E7136823F04E
:10D0100008031360FFF74BB87B780B2B00F2868078
:10D02000DFE803F006111C2733414C57626B737E17
:10D03000B978464A484852F821300068034442F81B
:10D040002130FFF734B8B978404A434852F82130CC
:10D0500000681B1A42F82130FFF729B8B9783B4A1B
:10D060003D4B52F821001B68434342F82130FFF743
:10D070001EB8B978354A384852F82130006893FB19
:10D08000F0F342F82130FFF712B8B9782F4A324B4B
:10D0900052F82140186894FBF0F300FB134342F868
:10D0A0002130FFF704B8B978284A2B4852F82130CC
:10D0B0000068034042F82130FEF7F9BFB978234AEF
:10D0C000254852F821300068034342F82130FEF72A
:10D0D000EEBFB9781D4A204852F82130006843401D
:10D0E00042F82130FEF7E3BF1B4BB9781B68174AA3
:10D0F000DB4342F82130FEF7DABF174BBA781968E4
:10D10000124B43F82210FEF7D2BFB9780F4A124BE8
:10D1100052F821001C6842F821401860FEF7C7BF92
:10D120000A4BBA7853F822200B4BE7E603230B7027
:10D13000FEF7BDBF7B780B2B00F29780DFE803F092
:10D140000E18222C37444E58626B737E080900205B
:10D15000E80800207007002004090020B84AB978C8
:10D16000B84B53F8213011680B441360FEF79FBF92
:10D17000B34AB878B349136851F820105B1A1360AA
:10D18000FEF795BFAE4AAF4BB97853F8211013683C
:10D190004B431360FEF78BBFA94AB878A9491368BF
:10D1A00051F8201093FBF1F31360FEF780BFA44AFF
:10D1B000A44BB978106853F8211090FBF1F301FBF0
:10D1C00013031360FEF773BF9D4AB9789D4B53F864
:10D1D000213011680B401360FEF769BF984AB97897
:10D1E000984B53F8213011680B431360FEF75FBF73
:10D1F000934AB978934B53F8213011684B40136030
:10D20000FEF755BFBA788F4B53F822308C4ADB4378
:10D210001360FEF74CBF8B4BBA7853F82220884B33
:10D220001A60FEF744BFB978864A854B52F8210050
:10D230001C6842F821401860FEF739BF814BBA786C
:10D2400053F822207E4B1B689A42FFF6B2AD7E4A0D
:10D2500013680BBF23F0060323F0050343F001031B
:10D2600043F002031360FEF722BF03230B70FEF7A7
:10D270001EBFB978734A52F82100184442F82100C1
:10D28000FEF715BFB9786F4A52F82100C01A42F86C
:10D290002100FEF70CBFB9786A4A52F821005843C2
:10D2A00042F82100FEF703BFB978664A52F8210020
:10D2B00090FBF3F042F82100FEF7F9BEB978614A1D
:10D2C00052F8214094FBF3F003FB104342F8213065
:10D2D000FEF7EDBEB9785B4A52F82100184042F8DB
:10D2E0002100FEF7E4BEB978564A52F821001843EF
:10D2F00042F82100FEF7DBBEB978524A52F821000D
:10D30000584042F82100FEF7D2BEB9784D4A52F893
:10D310002130DB4342F82130FEF7C9BEB978494AD3
:10D3200042F82130FEF7C3BEB978464A52F82120B0
:10D3300093428AE703232B70FEF7B9BE434B1B6869
:10D34000C7F80330FEF736F9FEF7B1BE3C4B1B6859
:10D35000BB703E4B1B68C7F80330FEF72BF9FEF796
:10D36000A6BEFBF7C7FE3A4B012283F8C020D7F8D0
:10D370000320C3F8C420FEF79ABE7878314951F8EB
:10D380002020013A002A41F820207EF790AE304A52
:10D39000C2F8C430FEF78BBE2C4B1B68C7F80330B5
:10D3A000FCF74EFE264B1B68A370284B1B68C4F885
:10D3B0000330FCF7B1FEFEF77ABE214B1B68BB7051
:10D3C000224B1B68C7F80330FCF73AFEFEF76FBE2E
:10D3D0001B4B1B78BB70FEF771BE194B1B68BB70F3
:10D3E000FDF7B0F9FEF763BE154B1B68BB70FBF78A
:10D3F000ABFEFEF75CBE124B1B68BB70134B1B6889
:10D40000C7F80330FDF79EF9FEF751BE0C4B1B68C1
:10D41000FF2B3EF64CAE0B4A52F823200B4B4A60D2
:10D420001A60094B2AB91A6842F008021A60FEF71E
:10D430003EBE1A6822F008021A60FEF738BE00BF2E
:10D44000040900200809002070070020E8080020D7
:10D4500078F6FF1FC84AD2F8C81007293EF627AE53
:10D4600078780C283EF623AEDFE810F00D001F00A0
:10D4700031004300550067007A008C009E00B00028
:10D48000C200D400E600BD48006804077EF50FAE78
:10D49000481C02EB8101C2F8C800D2F8C400C1F8F0
:10D4A000B001C2F8C430FEF702BEB44800680007FD
:10D4B0003EF5FDAD481C02EB8101C2F8C800D2F870
:10D4C000C400C1F8B001C2F8C430FEF7F0BDAB48EB
:10D4D0000068C7077EF5EBAD481C02EB8101C2F87E
:10D4E000C800D2F8C400C1F8B001C2F8C430FEF7D9
:10D4F000DEBDA2480068C6073EF5D9AD481C02EB68
:10D500008101C2F8C800D2F8C400C1F8B001C2F865
:10D51000C430FEF7CCBD9948006845077EF5C7AD1D
:10D52000481C02EB8101C2F8C800D2F8C400C1F85F
:10D53000B001C2F8C430FEF7BABD9048006810F0E0
:10D54000050F3EF4B4AD481C02EB8101C2F8C800DF
:10D55000D2F8C400C1F8B001C2F8C430FEF7A7BDCC
:10D560008648006884077EF5A2AD481C02EB810165
:10D57000C2F8C800D2F8C400C1F8B001C2F8C43083
:10D58000FEF795BD7D48006880073EF490AD481CCD
:10D5900002EB8101C2F8C800D2F8C400C1F8B001A2
:10D5A000C2F8C430FEF783BD74480068C7067EF534
:10D5B0007EAD481C02EB8101C2F8C800D2F8C4005D
:10D5C000C1F8B001C2F8C430FEF771BD6B48006805
:10D5D00086067EF56CAD481C02EB8101C2F8C800DE
:10D5E000D2F8C400C1F8B001C2F8C430FEF75FBD84
:10D5F0006248006845067EF55AAD481C02EB810181
:10D60000C2F8C800D2F8C400C1F8B001C2F8C430F2
:10D61000FEF74DBD5948006804067EF548AD481C2C
:10D6200002EB8101C2F8C800D2F8C400C1F8B00111
:10D63000C2F8C430FEF73BBD50480068C0057EF517
:10D6400036AD481C02EB8101C2F8C800D2F8C40014
:10D65000C1F8B001C2F8C430FEF729BD00F034FEB5
:10D66000FEF725BD00F031FEFEF721BD00F041FEC2
:10D67000FEF71DBD00F03EFEFEF719BD00F03BFEBB
:10D68000FEF715BD00F038FEFEF711BD7A782AB11D
:10D69000012A09D003230B70FEF709BD364B012286
:10D6A00083F8C020FEF703BDB3F5805FBEF40BAD79
:10D6B000314981F8C020C1F8C430FEF7F8BC2E4BC8
:10D6C000022283F8C020FEF7F2BC2D4A127D920799
:10D6D0000BD4B3F5805FBEF4F6AC274A042182F880
:10D6E000C010C2F8F831FEF7E2BC08230B70FEF759
:10D6F000DEBC214B002283F8C020FEF7D8BC214AB3
:10D70000214D012111701E4AB3F5805F9078287079
:10D7100027D2127D12EA010423D118466946FBF78D
:10D72000DDFB9DF800306B709DF80130AB709DF80B
:10D730000230EB709DF806302B719DF805306B714F
:10D740009DF80430AB719DF80330EB712C7201230E
:10D75000E95C2A7A01330A44082B2A72F8D1FEF7D1
:10D76000A6BC01230022EA540133082BFBD12B78FD
:10D770002B72FEF79CBC00BF78F6FF1F70070020DD
:10D780000C80FF1FEC080020ED080020A04B0122B8
:10D790001A70A04BA04A9B781370A04B1968002305
:10D7A0000139013311F8010FD054082BF9D1FEF7DC
:10D7B0007EBC0C22CA714B71F0220B238A710B7153
:10D7C000FEF775BC924B964801221A70914B924A13
:10D7D0009B781370002301331918082B11F8091CCA
:10D7E000D154F8D1FEF763BC7B78032B3EF65FACD7
:10D7F000DFE803F002101E238A4B93F8C020CA71A1
:10D8000093F8CC20D3F8F8318A711A0A4A710B7157
:10D81000FEF74DBC834B93F8C020CA7193F8CC201F
:10D82000D3F8C4308A711A0A4A710B71FEF73FBCF3
:10D830007D4B1B684B60FEF73ABC7C4B1B684B6012
:10D84000FEF735BC7A78002A7EF431ACBA78002A2B
:10D850007EF42DAC40F2D24293427EF428AC0021FB
:10D8600045F2FF70FBF7BBFAFBF746FB0120FAF726
:10D87000E1FFFEF71CBC7A786D4B9AB91A706D4ABD
:10D88000E3781370674A92F8FC116B4A11706B4988
:10D8900000220A706A490A706A4A11780B431370B1
:10D8A000FEF705BC0122E9E70422694645F2FB7058
:10D8B000FBF7E8FA009BD7F803209A4206BF012342
:10D8C0006B606E60FEF7F3BBBB782A2B07D1042296
:10D8D0005D4945F2FB70FBF794FAFEF7E8BB0323C2
:10D8E0000B70FEF7E4BB7A78032A47D8DFE802F032
:10D8F0001B0234424B4CD4F80002002104F50172A3
:10D9000081423EF4D4AB52F821509D4201F1010511
:10D9100020D102EB8503043B0138814214D3C4F8C3
:10D920000002FEF7C4BB3F4AD2F8001209299DBF8E
:10D93000481CC2F8000202EB8102092394BFC2F81E
:10D9400004322B70FEF7B3BB53F8042F43F8042CBA
:10D950000131E2E72946D3E7324A0023C2F8003218
:10D96000194602F5017242F8231001330A2BFAD14D
:10D97000FEF79DBB0A236B60FEF799BB03232B7058
:10D98000FEF795BB7B78812B7EF49DABBB78922B09
:10D990007EF499ABBB79A32B7EF495AB7B79B42B4A
:10D9A0007EF491AB3B79C52B7EF48DABFB78D62B07
:10D9B0007EF489ABFBF74FF9FAF760FE0446FAF7FD
:10D9C0005DFE001B0028B8BF4042B0F57A7FF6DB51
:10D9D000FAF72EFF1D4B00221A604FF0FF32C3F8FA
:10D9E0007021C3F87022C3F87421C3F87422C3F8FD
:10D9F0007821C3F87822C3F87C21C3F87C22144B29
:10DA0000144A1A600120FAF715FFFEF750BB00BF59
:10DA1000EC0800200C80FF1FED0800200880FF1F8D
:10DA20000080000078F6FF1FE808002004090020AD
:10DA3000CC030020F803002030070020EA03002078
:10DA400060070020CD0300206B07002010E000E0FD
:10DA50000080FF1F78563412F7B50F4C07460E466C
:10DA600094E803008DE803000C49C1F803300C4B27
:10DA70008A7000220F704E701A70FEF733F9094A4F
:10DA8000217882F80C119DE80300636884E80300A4
:10DA9000184603B0F0BD00BFFC0800206807002056
:10DAA000F708002078F6FF1FF7B504461F4A637891
:10DAB0001370A3785370E37893702379937163792B
:10DAC0005371A3791A4D1371E379D3700E4695E81B
:10DAD0000300184B00221A708DE80300FEF702F9CC
:10DAE000154B1A786F462B469AB9327072702A78A5
:10DAF000B2706A78F270EA793271AA7972716A79D1
:10DB0000B2712A79F27197E8030083E8030003B049
:10DB1000F0BD012AF7D10948721EF11D10F8014F1E
:10DB200002F8014F8A42F9D1EDE700BF68070020F3
:10DB3000FC080020F7080020EC080020ED08002079
:10DB40002DE9F043994B9A4C1B788FB06BB1994BF0
:10DB50001B78063BDBB2192B04D8974A22FA03F351
:10DB6000D90702D4002384F8FC3194F8FC31934E99
:10DB70005A1E012A51D89249012BCA68079214BF34
:10DB8000082307238DF81830327894F82D328DF859
:10DB9000193000238DF81A30002A33D18B688DF8A4
:10DBA0002030884B8DF8272019788DF8211059786E
:10DBB0008DF82210D9798DF8231099798DF82410D9
:10DBC00059791B798DF825108DF8263006A801F0BB
:10DBD000BFFE002800F028837B4B1A789846002A65
:10DBE00000F01E81794B7A4F1B78013B062B00F227
:10DBF0001381DFE813F0F100F10058011101110168
:10DC000011017F01012AE1D17248013306AA1A44A9
:10DC1000195CD171082BF8D1D8E7032B3DD13378AB
:10DC200083BBDFF89C81674F98F8020098F8015099
:10DC30003B7805441D447B781D44FB791D44BB792A
:10DC40001D447B791D443B791D44FAF751FD98F83A
:10DC50000100FAF74DFD3878FAF74AFD7878FAF7BF
:10DC600047FDF879FAF744FDB879FAF741FD78797C
:10DC7000FAF73EFD3879EDB2FAF73AFD2846FAF7A1
:10DC800037FDA9E7012BA7D1524F0025785D01355B
:10DC9000FAF72EFD092DF9D19EE7042B2BD1484F21
:10DCA000DFF82081B8787D780023012205441544EF
:10DCB00088F8013088F80020C8F80430FAF718FD19
:10DCC0007878FAF715FD98F80000FAF711FD98F842
:10DCD0000100FAF70DFD98F80700FAF709FD98F82A
:10DCE0000600FAF705FD98F80500FAF701FDEDB218
:10DCF00098F80400C0E7072B37D1337853BB304B7B
:10DD00009F7893F801802F4B8DF800701D7858781C
:10DD1000D9798DF8025047443D449A798DF8030033
:10DD2000284493F805C08DF80410014493F804E0EA
:10DD30008DF805200A440CEB020373448DF8018032
:10DD40008DF806C08DF807E08DF808306846FAF7C0
:10DD50007FFF41E7012BF9D11E4900235A5C0DF8E2
:10DD600003200133092BF9D1F0E7082B7FF434AFFE
:10DD7000144A1349002301205370107053608A78AD
:10DD800049788DF800200A4402448DF801108DF87E
:10DD900002008DF803308DF804308DF805308DF8D1
:10DDA00006308DF807308DF80820CFE7F608002000
:10DDB00078F6FF1F6807002011020002EC0800201F
:10DDC0000C80FF1FFC0800206007002030070020A7
:10DDD000EA030020ED080020B14A397893688DF8F5
:10DDE000303080238DF831308A238DF83230002393
:10DDF0008DF833308DF834308DF835308DF836109D
:10DE00008DF8293007218DF82A300AA8D3688DF8BB
:10DE100028100B9301F09CFD00233B7088F8003024
:10DE2000002384F8FC31337094F82C3213B10120B4
:10DE3000FAF700FD06A801F017FD0646002800F0DD
:10DE40004781984B9DF820201A709DF821205A7028
:10DE50009DF822209A709DF823209A719DF8242025
:10DE60005A719DF825201A719DF82620DA709DF8C8
:10DE7000193084F82D32FAF701FC8B4B18608B4B6C
:10DE800000221A709DF81830072B0CBF01230223C3
:10DE900084F8FC3194F8C0305A1E012A4AD9052B67
:10DEA00048D0012247E0DFF8F8913B7899F802006A
:10DEB00099F8015005440A351D44FAF719FC99F800
:10DEC0000100FAF715FC8020FAF712FC8A20FAF715
:10DED0000FFC0020FAF70CFC0020FAF709FC0020E8
:10DEE000FAF706FCEDB23878FAF702FC2846FAF7A2
:10DEF000FFFB91E76A4A507893788DF80C303A78B6
:10DF00008DF80D00802103448DF80E100A338A210C
:10DF10008DF80F101344002103A88DF810108DF810
:10DF200011108DF812108DF813208DF81430FAF7B7
:10DF30008FFE71E700225E4B1A7094F8C030042BFC
:10DF400004D1584B19780A0640F1718194F8FC21EC
:10DF5000082A04D840F25113D340DF0701D4FDF75B
:10DF6000C1FE94F8FC31092B74D1FAF787FBD4F881
:10DF7000F430504DC01A00282A68B8BF4042904281
:10DF800009D94D4B1A78012A04BF02221A70FAF7F8
:10DF900075FBC4F8F400FAF771FBD4F8F8306A683E
:10DFA000C01A0028B8BF4042904209D9424B5A7863
:10DFB000012A04BF02225A70FAF760FBC4F8F80085
:10DFC000FAF75CFBD4F8FC30AA68C01A0028B8BF86
:10DFD0004042904209D9384B9A78012A04BF022264
:10DFE0009A70FAF74BFBC4F8FC00237893B363787C
:10DFF00083BB314A31481D46D15C022940F00B8178
:10E0000050F823104E1C00F005812D4A84F8F4319D
:10E010001268C4F8D8212B4A1268C4F8DC21D4F85D
:10E02000C420C4F8E021284AC4F8C4101268C4F817
:10E03000E42194F8CC20C4F8E8210023D4F8D421BA
:10E04000C4F8EC2184F8CC30D4F8D021C4F8F02105
:10E050000123637094F8FC31092B06D194F8C02099
:10E06000022A04BF052284F8C020D4F80022002A26
:10E0700000F0DA80092B40F0D78094F8C030012BF3
:10E0800040F0D280D4F8C4101048002350F8235038
:10E090008D4240F0C580052384F8C030C4E000BF45
:10E0A0000C80FF1F6807002020070020BC03002011
:10E0B000F7080020E0060020310700207CF6FF1F53
:10E0C000E808002004090020700700207CF8FF1FEA
:10E0D00003A8FAF725FB054600284ED0FAF738FBCF
:10E0E00008B184F82E6294F82E229DF80C10531C6F
:10E0F000DBB22244092B84F82E3282F82F127FF4EF
:10E100001CAF604A94F82F1252780023914284F891
:10E110002E327FF412AF5C495A5C01331644082B4F
:10E12000F6B2F9D194F83732B34222D1574B94F872
:10E1300030221A7094F831225A7094F832229A7070
:10E1400094F833229A7194F834225A7194F8352253
:10E150001A7194F83622DA70FAF790FA4C4B4D4A5D
:10E16000186000231370032284F8FC2184F82E32F7
:10E1700090E6042384F8FC31DFE60AAE3046FAF775
:10E1800054FD48B32B46F25C01331544082BEDB225
:10E19000F9D19DF83020AA42ECD13C4B9DF82920C2
:10E1A0001A709DF82A205A709DF82B209A709DF8BD
:10E1B0002C209A719DF82D205A719DF82E201A71ED
:10E1C0009DF82F20DA70FAF759FA314B1860314B6D
:10E1D00000221A7007235BE694F8C030013B012B44
:10E1E0003FF6ABAED4F8C430B3F5805F0ED2FAF789
:10E1F000F7FC58B1D4F8C4002449431CC4F8C43017
:10E20000FAF76CFE092384F8FC314AE6002384F80F
:10E21000C03092E6D55401332F2B7FF4EDAE19E7D1
:10E2200001339A427FF432AF0FB0BDE8F08394F827
:10E23000FC01082804D840F25112C240D207F3D49E
:10E24000D4F8F801144DD3F803306970B0F5805F4D
:10E250006B6012D20D49FAF72DFE0C49D4F8F80183
:10E26000FAF77EFE38B1D4F8F8310133C4F8F8314A
:10E2700065232B70D8E70723FBE707232B700023C8
:10E280000AE700BF0C80FF1FA7F8FF1F68070020E8
:10E29000280700202F070020FC080020704710B539
:10E2A000074CFAF7EBF92368C01AB0F5FA7F05D9E5
:10E2B000044B0222DA60FAF7E1F9206010BD00BFDA
:10E2C000080D002000F00F407047064B5A7832B915
:10E2D000D3F80310044B01B901221A7070470322CE
:10E2E000024BFAE768070020E3030020FC08002047
:10E2F000704770477047704770477047024B185C13
:10E30000431F584258417047B0F8FF1F73B5144C73
:10E3100023180646DB780D4623B94FF0C05207217B
:10E3200002F0EEF90F4A602303FB062301229B7DD6
:10E33000019285EAE572A2EBE572D2B20092062163
:10E340000022304602F03EF9002D04EB060304EBF8
:10E350008604B4BF01220222DA70A56002B070BD4B
:10E36000B0F8FF1FB4050020184B1A1873B5D17808
:10E37000044641B303EB80030025D57007214FF01D
:10E3800080529D6002F0AEF94FF0006207212046F6
:10E3900002F0B6F960230E4A6343D618D35C93B1FA
:10E3A0005021204602F05EF921210246204602F06B
:10E3B00033F9327DB37D0192727D009206212A46A7
:10E3C000204602F0FFF802B070BD00BFB0F8FF1F9A
:10E3D000B40500202DE9F347174D2C7D05F11508F4
:10E3E0004CB9E0B2FAF738FB08F804000134082C05
:10E3F000F7D101232B75DFF848A0104F2724002602
:10E400004FF00209F0B2FAF727FB18F80630834202
:10E410001DD006F1080308F806005AF82330022B35
:10E4200010D0032B02D0012B11D180B13B5D012B09
:10E4300008BF07F804900AE0B0F8FF1F310700207A
:10E44000E006002018B93A5D012A00D13B5501369B
:10E45000082E04F10104D5D1B04CE369C3B1B04E2C
:10E460003778AFB9FAF70AF9AE4B1B68C01A002823
:10E47000E369B8BF404298420AD9384602F088F9A9
:10E48000012002F085F9022002F082F901233370A5
:10E49000236AC3B1A44E3778AFB9FAF7EFF8A34BAC
:10E4A0001B68C01A0028236AB8BF404298420AD9A4
:10E4B000384602F06DF9012002F06AF9022002F0FC
:10E4C00067F9012333702221687F994E02F0CAF860
:10E4D0008046687F02F043F90F210446687F02F00E
:10E4E000C1F80746687F06EBC0131B69002B00F0DC
:10E4F0000781002B88EAE872A2EBE872B8BF5B42A2
:10E50000B3EB022F80F2FC802B189B7F43B94FF0B6
:10E510008062012102F0E6F86B7F01222B449A779A
:10E5200004F00903092B31D1687F8249C21C8B5C3E
:10E53000DBB2012B0ABF4FF0020E8B5C01F802E048
:10E540007D490A7818BFB3FA83F342FA00FE18BF78
:10E550005B091EF0010F15D04FF0010CDFF8FC91A4
:10E560000CFA00FE89F800E0DFF8F49189F800C0A9
:10E57000DFF8F0C19CF800C0BCF1000F02D122EA24
:10E580000E020A7013B1092102F0F6F8A10010D5AD
:10E59000687F684A00F10F03D15C012904BF0221A2
:10E5A000D1544FF0005102F0E7F86B7F634A01212C
:10E5B000D154220507D5B8F1000F04D14FF4006102
:10E5C000687F02F0D9F8E30407D5B8F1000F04D151
:10E5D0004FF48051687F02F0CFF8A00407D5B8F15E
:10E5E000000F04D14FF40051687F02F0C5F86104B8
:10E5F00007D5B8F1000F04D14FF48041687F02F0D5
:10E60000BBF8687F06EBC0131B6A0BB362031FD510
:10E6100002F0BEF85021687F02F024F86B7F484A70
:10E6200052F823202121821A184601F0F5FF4FF4F9
:10E630008021687F02F0A0F86B7F3E4903F115024C
:10E64000885C012804BF022088543E4A0121D1542D
:10E650006B7F17F0800105EB030200F0858092F8D4
:10E66000211089B9012182F82110374A1A44127EFB
:10E6700012F0010F08D002211B2211FB03232D4AA7
:10E68000D05C012808BFD1546B7FEA1817F480775B
:10E6900092F8241074D089B9012182F824102A4AF2
:10E6A0001A44D27E12F0010F08D00E33214A12F81C
:10E6B0001310012904BF022102F81310F9F7DEFF3D
:10E6C000AB6AC01A0028B8BF40420A2840F39580C0
:10E6D000687F1E4B1E4A1F491F4F0344024401EB33
:10E6E000800101F000FF6C7F2A5D6023052A6AD853
:10E6F000DFE812F050008600CE001301250167010B
:10E700002B189B7F002B3FF40BAF4FF08062012151
:10E7100001F0F6FF6B7F00222B4400E70C80FF1F07
:10E720002F07002028070020BC030020200700201E
:10E730003004002031070020F803002028040020C6
:10E74000EC030020E4030020E00600202B0400205E
:10E75000E0030020FC030020B4050020EA030020B1
:10E7600060070020CC03002092F8210000288BD005
:10E7700082F82110C24A1A44127E12F0020F79E781
:10E7800000299BD082F82470BD4A1A44D27E12F030
:10E79000020F89E76343FB5CABB1204600F0B2FE99
:10E7A00088B91021204606EBC41601F095FB737A58
:10E7B00020F4F852DB0842EA03221021204601F03F
:10E7C00045FB01232B55687F00F092F96C7F602395
:10E7D0006343FB5C3BB12B19DB78012B00F03C81E0
:10E7E000022B00F045816B7F0133DBB2022B88BF27
:10E7F00000236B77F9F742FFA86202B0BDE8F0870B
:10E8000000220521204601F007FF602202FB04726E
:10E810002046117D937D0191527D009206210022B8
:10E8200001F0D0FE7921204601F01CFF7F281BDC7F
:10E83000C0F1800604222021204601F0EDFE914A1D
:10E840002421204601F0E8FE2121204601F00AFFA4
:10E8500037218219204601F0DFFEF9F70FFF05EBA3
:10E860008403D8620223ADE7B0F5C07F02DAC0F5B9
:10E87000C076DFE7B0F5207F02DAC0F52076D9E771
:10E88000B0F5607FB4BFC0F56076C0F59066D1E7A3
:10E89000F9F7F4FE05EB8403DB6AC01A0028B8BF61
:10E8A0004042B0F57A7F8EDD06EBC416F66956B1AC
:10E8B0002121204601F0D6FE50210246204601F0DB
:10E8C000ABFE03237EE732462021204601F0A4FE62
:10E8D00032462421204601F09FFE5021204601F0BF
:10E8E000C1FE21210246204601F096FE212120464C
:10E8F00001F0B8FE37210246204601F08DFE0422C9
:10E900002021204601F088FE5E4A2421204601F0A5
:10E9100083FE5D4B01221A55D3E74FF0C052072109
:10E92000204601F0EDFE594A0721204601F0DAFEAB
:10E93000F9F7A4FE05EB8403D862042342E7F9F754
:10E940009DFE05EB8403DB6AC01A0028B8BF404275
:10E95000B0F57A7F7FF737AF06EBC4164FF0194258
:10E960000721204601F0CCFE737E0BB11B0725D595
:10E970004FF020620721204601F0B4FE80220521DD
:10E98000204601F049FE5921204601F06BFE60232C
:10E9900003FB0473002218613D4B5021204643F8CD
:10E9A000242001F05FFE21210646204601F05AFE98
:10E9B000384B301A43F82400052303E74FF0007268
:10E9C000D8E7634317F80380B8F1000F7FF4FBAE7C
:10E9D0002046FFF7C9FC06EBC4164FF0046207217E
:10E9E000204601F08DFE03220521204601F014FE91
:10E9F000B37DB27A0193737A009306214346204691
:10EA000001F0E0FD1021204601F066FA102140F4EB
:10EA1000F852204601F01AFAF37D05F80480CBB9CC
:10EA200001222021204601F0F7FD0022242120466A
:10EA300001F0F2FD2121204601F014FE144B53F8A1
:10EA400024202121821A204601F0E6FD0E4B0122EE
:10EA50001A55B8E60222E4E75021204601F002FEF2
:10EA6000A0F5C332A03A2121204601F0D5FDBAE637
:10EA70005021204601F0F6FD00F5C332A032F2E746
:10EA8000E006002040420F00E70300200000408124
:10EA9000D4030020EC030020024B03EB80008068CD
:10EAA000704700BFB0F8FF1F38B5104B03EBC01321
:10EAB0000446DB7D0D46B3B90122202101F0ACFDF7
:10EAC00020464FF08052072101F00CFE20464FF007
:10EAD0000062072101F014FE2A4620462421BDE8E9
:10EAE000384001F099BD0222E7E700BF3004002062
:10EAF0002DE9F74F04469A4DE6010F2101F0B2FDD2
:10EB0000A919020A0B7AD1F8048013F0400F14BF40
:10EB1000A95955F806A04FEAD01015BF02F0010B15
:10EB200000F0010B00F0010202F001021CBFC1F174
:10EB3000000AC8F100081F0603F03F0900922046B2
:10EB400013D501F031FFB0FA80F35B0909F1FF3111
:10EB5000009A072972D8DFE811F00E000E000E00AF
:10EB60000E00BD02BD02BD02BD0201F01DFF031C6F
:10EB700018BF0123EAE77B4F3B5D013B0E2B5DD8BD
:10EB8000DFE813F00F0039005F006B009000AD006C
:10EB9000D000F8006201F001F6015C005C027E0228
:10EBA0006502DFF8CCB1704B4FF000084FF0010A5E
:10EBB0005FFA88F0844209D0AA1992F84E2072B107
:10EBC00005EBC81191F84E10914208D10121009334
:10EBD00001F048FD009B4BF8280008F803A008F15D
:10EBE0000108B8F1030FE3D1A9F10209B9F1010F4E
:10EBF00030D802232FE007EB840301215A68204616
:10EC000042F0020201F008FD4FF000082E445FFAC6
:10EC100088F0844208D096F84E3043B105EBC81214
:10EC200092F84E209A4202D15146FFF73DFF08F17B
:10EC30000108B8F1030FEAD107F8048003B0BDE87A
:10EC4000F08F002AFAD02121204601F00BFD474B1E
:10EC500043F8240004233B55F0E707EB840301212C
:10EC60005A68204642F0010201F0D6FC4FF000083D
:10EC7000CAF1000A2E445FFA88F0844208D096F860
:10EC80004E3043B105EBC81292F84E209A4202D1A1
:10EC90005146FFF709FF08F10108B8F1030FEAD167
:10ECA0000523D8E7BBF1000FC8D04FF000082E4471
:10ECB0005FFA88F3A34208D096F84E3043B105EBD3
:10ECC000C81292F84E209A4202D1404601F060FDEF
:10ECD00008F10108B8F1030FEAD10623BBE707EBFF
:10ECE000840301215A68204622F0030201F094FCBB
:10ECF0004FF000092E445FFA89F0844208D096F85C
:10ED00004E3043B105EBC91292F84E209A4202D11F
:10ED10004146FFF7C9FE09F10109B9F1030FEAD134
:10ED2000072398E7BBF1000F88D1C8F100082E44F3
:10ED30005FFA8BF0844208D096F84E3043B105EB71
:10ED4000CB1292F84E209A4202D14146FFF7ACFE18
:10ED50000BF1010BBBF1030FEAD108237BE700BFE6
:10ED600030040020E8F8FF1FE7030020C003002064
:10ED7000ECF8FF1FBBF1000F3FF460AF21212046EC
:10ED800001F070FC4FF00009834605EB060A5FFABC
:10ED900089F0844208D09AF84E3043B105EBC9128D
:10EDA00092F84E209A4202D10021FFF77DFE09F130
:10EDB0000109B9F1030FEAD1C04A52F82430A3EB9C
:10EDC0000B0342F8243007EB840301215A682046E4
:10EDD00022F0030201F020FC4FF0000A5FFA8AF9EA
:10EDE0004C4509D0AB1993F84E3023B305EBCA124A
:10EDF00092F84E209A421ED105EBCA13DB7D0BBB65
:10EE000005222021484601F007FC424624214846BD
:10EE100001F002FC4FF080520721484601F070FCDF
:10EE20004FF000620721484601F05CFC5A4637214A
:10EE3000484601F0F1FB0AF1010ABAF1030FCDD106
:10EE4000092308E70622DCE70F21204601F00AFC2F
:10EE5000C1077FF5F3AE2121204601F003FC984B5A
:10EE600043F824004FF0000A05EB060B5FFA8AF026
:10EE7000844208D09BF84E3043B105EBCA1292F899
:10EE80004E209A4202D10021FFF70EFE0AF1010A3C
:10EE9000BAF1030FEAD14FF0000A5FFA8AFB5C4532
:10EEA00009D0AB1993F84E30F3B105EBCA1292F8C2
:10EEB0004E209A4218D1602303FB0AF3814A9B5CDF
:10EEC000CBB35021584601F0CDFB7F4B212143F8B5
:10EED0002A00584601F0C6FB7C4B024643F82A0044
:10EEE0003721584601F098FB0AF1010ABAF1030FE5
:10EEF000D3D1A9F10309B9F1010F00F2A6804FF0B7
:10EF00000009C8F100082E445FFA89F0844208D055
:10EF100096F84E3043B105EBC91292F84E209A4252
:10EF200002D14146FFF7C0FD09F10109B9F1030F14
:10EF3000EAD10A238FE61A4637215846009301F09A
:10EF40006BFB009B21211A46584601F065FB009B94
:10EF500050211A46584601F05FFB5B4A009B42F87D
:10EF60002A30C1E7BBF1000F3FF468AE0B2372E615
:10EF7000BBF1000F7FF462AE2121204601F072FB4D
:10EF800005EB060982465FFA8BF0844208D099F8B7
:10EF90004E3043B105EBCB1292F84E209A4202D18B
:10EFA0000021FFF781FD0BF1010BBBF1030FEAD14B
:10EFB000DFF81CB102239AFBF3F34FF0000A009331
:10EFC0005FFA8AF94C4509D0AA1992F84E2062B32B
:10EFD00005EBCA1191F84E10914226D15BF82A2018
:10EFE000012122F00302484601F016FB05EBCA128C
:10EFF000D27D0ABB05222021484601F00DFB424686
:10F000002421484601F008FB4FF080520721484672
:10F0100001F076FB4FF000620721484601F062FBE9
:10F02000009A3721484601F0F7FA0AF1010ABAF1CD
:10F03000030FC5D10D230EE60622DCE70F21204683
:10F0400001F010FBC2077FF5F9AD0E2303E64FF088
:10F0500000082E445FFA88F0844208D096F84E30BB
:10F0600043B105EBC81292F84E209A4202D100211A
:10F07000FFF71AFD08F10108B8F1030FEAD1E4E740
:10F08000DFF84C904FF000082E445FFA88F084427D
:10F0900008D096F84E3053B105EBC81292F84E20C6
:10F0A0009A4204D159F82820012101F0B5FA08F15B
:10F0B0000108B8F1030FE8D10023CCE5C00300201C
:10F0C000D4060020B4050020EC030020D403002067
:10F0D000ECF8FF1FC54F395D01390E293FF6AEAD83
:10F0E00001A050F821F000BF25F100007DF10000E3
:10F0F000DDF10000FDF1000061F200003DEC0000D8
:10F100007FF200003DEC00003DEC000033F3000016
:10F1100049F30000D7F20000F9F300009FF400006B
:10F120006DF40000DFF8CCA2B14B4FF000084FF0B7
:10F13000010B5FFA88F0844209D0AA1992F84E2098
:10F1400072B105EBC81191F84E10914208D108F840
:10F150000AB00121009301F085FA009B43F82800D2
:10F1600008F10108B8F1030FE3D1B9F1060F3FF43C
:10F1700040ADB9F1080F7FF46DAD3AE5B9F1060F76
:10F1800023D107EB84035A6822F0030242F0020203
:10F190000121204601F040FA4FF000082E445FFAAA
:10F1A00088F0844208D096F84E3043B105EBC8127F
:10F1B00092F84E209A4202D15146FFF775FC08F1B1
:10F1C0000108B8F1030FEAD136E5B9F1080FE3D130
:10F1D00007EB84035A6822F00302D9E7A9F105017D
:10F1E000012906D82AB1B9F1060F3FF433AD0F2338
:10F1F00031E5002B3FF422AD0C232CE5B9F1050FCE
:10F2000025D107EB84035A6822F0030242F0010281
:10F210000121204601F000FA4FF00008CAF1000A6F
:10F220002E445FFA88F0844208D096F84E3043B1FD
:10F2300005EBC81292F84E209A4202D15146FFF7D0
:10F2400033FC08F10108B8F1030FEAD128E5B9F160
:10F25000070FE1D107EB84035A6822F00302D7E7D6
:10F26000A9F10502012A06D8BBF1000F03D0B9F1BC
:10F27000050FBCD1BDE4002B3FF4E0AC50E5002B02
:10F280007FF4DCACA9F10709B9F1010F0AD907EB4A
:10F29000840301215A6822F0030242F00202204650
:10F2A00001F0BAF94FF000092E445FFA89F0844268
:10F2B00008D096F84E3043B105EBC91292F84E20B3
:10F2C0009A4202D14146FFF7EFFB09F10109B9F17A
:10F2D000030FEAD12DE6002B7FF4B0ACA9F10709AA
:10F2E000B9F1010F0AD907EB840301215A6822F012
:10F2F000030242F00102204601F08EF94FF00009AE
:10F30000C8F100082E445FFA89F0844208D096F8CC
:10F310004E3043B105EBC91292F84E209A4202D109
:10F320004146FFF7C1FB09F10109B9F1030FEAD129
:10F33000FFE5002B3FF482AC2121204601F092F939
:10F3400007EB8403186111E6002B7FF477AC2121D1
:10F350002046019301F086F9019B00909A4607EB45
:10F36000840B5FFA8AF94C4509D0AA1992F84E200D
:10F370009AB305EBCA1191F84E1091422DD11C4B56
:10F3800053F82A20012122F00302484601F044F9F3
:10F3900005EBCA12D27D32BB05222021484601F07E
:10F3A0003BF942462421484601F036F94FF080529D
:10F3B0000721484601F0A4F94FF0006207214846B2
:10F3C00001F090F9DBF81020009B02211A44484616
:10F3D00092FBF1F2372101F01FF90AF1010ABAF1AB
:10F3E000030FBED126E60622D7E700BFE8F8FF1FCD
:10F3F000ECF8FF1FE70300200F21204601F032F94F
:10F40000C3077FF51BAC0E23212120463B5501F09D
:10F4100029F9314BDFF8C49043F8240000275FFA44
:10F4200087F8444509D0AB1993F84E30CBB105EBC2
:10F43000C71292F84E209A4213D100214046FFF79E
:10F4400033FB00223721404601F0E6F8002221215B
:10F45000404601F0E1F85021404601F003F949F837
:10F4600027000137032FDAD1FFF7E8BB4FF0000880
:10F470002E445FFA88F0844208D096F84E3043B1AB
:10F4800005EBC81292F84E209A4202D10021FFF7F4
:10F490000BFB08F10108B8F1030FEAD1D5E5DFF85D
:10F4A00040904FF000082E445FFA88F0844208D064
:10F4B00096F84E3053B105EBC81292F84E209A429E
:10F4C00004D159F82820012101F0A6F808F101081B
:10F4D000B8F1030FE8D1EFE5D4060020EC030020DB
:10F4E000ECF8FF1F024B1A5C0AB901221A5470474C
:10F4F000E8F8FF1F024B1A5C0AB10F221A5470473A
:10F50000E8F8FF1F014B185C704700BFE8F8FF1FC9
:10F51000764B774841F2300C2DE9F04F53F80C2030
:10F52000744FDFF8E4E142F0006243F80C2041F24E
:10F530003C0403F582511A5942F000621A510A68DC
:10F5400042F002020A601A5942F002021A514FF0C8
:10F550000C0A00224FF00409B823C0F808A0C260CA
:10F560004262C0F82090BB70634B03F5825141F2B8
:10F570004405C1F800E00121595341F24C056FF0F8
:10F5800006065E5141F250055C4E585141F254005E
:10F5900041F25E051A5241F258006FF00D081A5000
:10F5A00041F248004FF4087B19500720585341F2AC
:10F5B00056050EF1070E585341F24600504D1A52AF
:10F5C00041F25C001952A920F87003F583500560E0
:10F5D00041F2640002251A5241F26C001A5041F2C5
:10F5E00070001E5041F274000E361D5241F2780038
:10F5F00043F8008041F2680041F27E081D5048F255
:10F60000074023F8080041F2760823F8080041F289
:10F61000660040F2011823F8008041F27C0023F8D4
:10F6200000B00320D8763748C0F808A04FF0570A3A
:10F63000C2604262C0F800A0C0F820904FF0B60946
:10F6400087F8009003F58059C9F800E041F2040EF4
:10F650004FF0FF3923F80E1041F20C0E43F80E90D4
:10F6600041F2100E43F80E0041F214001A5241F21A
:10F6700018001A5041F20800195041F21E001952A8
:10F6800041F21600195241F206001A5241F21C00D2
:10F690001952A820787003F5815007F5D03710373C
:10F6A000076041F224001A5241F22C001A5041F234
:10F6B000340243F80C609D5241F238026FF00100B1
:10F6C000985041F2280241F23E009D5048F201025A
:10F6D0001A5241F236001A5241F2260223F80280F1
:10F6E00020221A53D976BDE8F08F00BF0070044085
:10F6F00000B00B40001002400080004004F9FF1FE2
:10F7000010B00B4000B003404C80FF1F0C282DD8D8
:10F71000DFE800F0070B0E112C2C2C2C142C1A24D3
:10F720002900134BD88880B27047114B1889FAE72B
:10F730000F4B5889F7E70E4B9889F4E70C4B588824
:10F7400083B240F2732003E0094B988883B28E2085
:10F7500058434FF6FF7390FBF3F07047044B188843
:10F7600083B24220F4E7024BD889E9E700207047D2
:10F7700004F9FF1F30B52E4D41F23C042B5943F0E4
:10F7800010032B512B4B4FF400741C636FF4F8756E
:10F790005C63A3F51433A4F13E542C441C604FF475
:10F7A00000545C60244C1C601C68E401FCD50138EA
:10F7B000072834D8DFE800F0312F2D2B2933270418
:10F7C0001E4858601E4B002058631E4818601E4893
:10F7D0004FF0806400EA8145C3F88040C3F884504C
:10F7E000FAB100EA8240C3F89040C3F894004FF0A9
:10F7F0008460C3F8A000C3F8A410AAB1C3F8B00095
:10F80000C3F8B42030BD1148DBE71148D9E71148EF
:10F81000D7E71148D5E71148D3E71148D1E7114898
:10F82000CFE7C3F89020E2E7C3F8B02030BD00BFB7
:10F8300000700440009004400F0080508720FE01BB
:10F84000004002400F0080000000FC1F8720FE03E4
:10F850008720FE0F8720FE138720FE278720FE6368
:10F860008720FEC78720FE07384AD2F88030C3F3CE
:10F870000363022B5FD0D2F89030C3F30363022BF3
:10F880005BD0D2F8A030C3F30363022B06D0D2F8CA
:10F89000B030C3F30363022B56D103231B0103F1E2
:10F8A000402202F50032D2F88010C1F3034101700A
:10F8B000D2F8801011F4801118BF01218170D2F8A4
:10F8C000801011F4001118BF012141704178B1BBC3
:10F8D000D2F88410C1F38A4103F1402303F50033C9
:10F8E0004160D3F88810090E0172D3F88810090C12
:10F8F0004172D3F88810090A8172D3F88810C17256
:10F90000D3F88C10090E0173D3F88C10090C4173D5
:10F91000D3F88C10090A8173D3F88C30C373D2F8F2
:10F9200080309B024CBF4FF084634FF08063C2F87D
:10F930008030012070470023B0E70123AEE7D2F802
:10F94000841021F06041C7E700207047004002406A
:10F95000184AD2F87031C3F303630C2B10B527D0CB
:10F960004478436804B3C3F31103C2F87431836865
:10F97000104A1BBAC2F87831C3681BBAC2F87C318E
:10F980008378002C14BF4FF042624FF040620BB1FD
:10F9900042F4801203781B0403F470231343054AD6
:10F9A0000120C2F8703110BD034901EA8343DCE74E
:10F9B000002010BD004002400000FC1F0B4B4FF028
:10F9C0000062C3F870214FF48022C3F87421084A02
:10F9D000C3F878216FF48471A2F166320A44C3F847
:10F9E0007C21044AC3F87021704700BF00400240E8
:10F9F000785634120000080C10B53A4BDA7842F011
:10FA00000202DA70384A1078C0B20228114641D09A
:10FA1000032835D0012832D1546891688C4215D220
:10FA2000D978C90707D45168D0684C1C5460425C2F
:10FA3000D2B21A7110BD997801F0DF0199709978EE
:10FA400001F0EF0199701074002317E0517C01F070
:10FA5000FF0049B9997801F0DF019970997801F0B8
:10FA6000EF019970107010BD997841F00401997000
:10FA7000917CC9B21971002353740323137010BD14
:10FA8000997801F0EF0199701B795169DBB20B7025
:10FA90000223F3E79469D06984421DD2D269886950
:10FAA000121A012A05D19A7802F0DF029A70002317
:10FAB0000B70CB698A699B1A022B9FBF094A937806
:10FAC00043F0080393708A694869531C8B61054BA6
:10FAD0001B79DBB2835410BD997801F0DF01997076
:10FAE000B2E700BF0070064014F9FF1F41F2340274
:10FAF0000A498B5843F080038B50094B4FF418721E
:10FB00009A62DA6203F5E0331B225A70C0229A70BF
:10FB100000225A71192000F081BF00BF007004401C
:10FB200000B0044010B5104B00241C745C749A6043
:10FB300001225C601A700D4AD960917801F0F701DA
:10FB40009170917841F010019170917800F0FE0071
:10FB500041F02001917010711A78002AFCD1187CB4
:10FB6000B0FA80F0400910BD14F9FF1F0070064084
:10FB700010B5104B00241C745C74DA6103229C6184
:10FB80001A700D4A5961917801F0F70191709178DE
:10FB900041F010019170917840F0010041F0200196
:10FBA000917010711A78002AFCD1187CB0FA80F09C
:10FBB000400910BD14F9FF1F0070064070B5144CC9
:10FBC000002563610126049B25746674A26065604C
:10FBD000E36140EA0603A561A3740E4BE160267061
:10FBE0009A7802F0F7029A709A7842F010029A70AE
:10FBF0009A7800F0FE0042F020029A701871237883
:10FC0000002BFCD1207CB0FA80F0400970BD00BF11
:10FC100014F9FF1F007006402DE9F3411C4F1D4CE5
:10FC200000264FF00C08F5B20423B7F84C20CDF8AD
:10FC300000800A21284600F071FD4FF48052002117
:10FC4000284600F0E9FCFA695421284600F0E4FC5B
:10FC500000225021284600F0DFFC626CFF210823BF
:10FC600084F8401084F84130019100936321D3B2AD
:10FC70002846C2F30722013600F0A4FC032E07F148
:10FC8000800704F16004CED102B0BDE8F08100BF6E
:10FC900030040020B405002038B50D460721044685
:10FCA00000F0E0FCEA074CBF40F0800220F0800248
:10FCB000AB074CBF42F4807222F4807268074CBFDD
:10FCC00042F0100222F0100229074CBF42F40072E9
:10FCD00022F40072EB064CBF42F0040222F0040250
:10FCE000A8064CBF42F0080222F0080269064CBF89
:10FCF00042F0200222F020022B064CBF42F04002CC
:10FD000022F04002E8054CBF42F0020222F002025B
:10FD1000A9054CBF42F4806222F480626B05204644
:10FD20004CBF42F4006222F400620721BDE8384073
:10FD300000F072BC072108B500F094FCC0F3C013BA
:10FD4000C10548BF43F00203C20648BF43F00403A5
:10FD5000810548BF43F00803420748BF43F0100342
:10FD6000010748BF43F02003820648BF43F0400329
:10FD7000410648BF43F08003820748BF43F48073C5
:10FD8000410548BF43F40073020548BF43F4806354
:10FD9000184608BD2DE9F34701F07F07352F0546CA
:10FDA000894692461C469DF828809DF82C6016D105
:10FDB00043EA022448EA042446EA0424224A9F3003
:10FDC00024F4736424F0030452F82030E404E40CB7
:10FDD00023EA040442F8204002B0BDE8F0876FF047
:10FDE00000720C2100F018FC0E21284600F03AFCAD
:10FDF0004FF0FF320C21284600F00EFC49F0800342
:10FE0000019300231A4600936D21284600F0DAFB87
:10FE10000196CDF80080234652466C21284600F01A
:10FE2000D1FB0E21284600F01DFC8301F9D544EAE0
:10FE30000A2407EB470048EA04242844024B46EA18
:10FE4000042443F82040C7E734F9FF1FF7B501F059
:10FE50007F05352D04460F4616460FD11D4A9F34A7
:10FE600026F4736626F0030652F82430F604F60CE6
:10FE700023EA060342F8243003B0F0BD6FF00072AD
:10FE80000C2100F0C9FB0E21204600F0EBFB4FF0E7
:10FE9000FF320C21204600F0BFFB47F08007002313
:10FEA0001A466D2120460197009300F08BFB3246E5
:10FEB0006C21204600F0B0FB0E21204600F0D2FB62
:10FEC0008301F9D505EB45052C44024B43F824602A
:10FED000D2E700BF34F9FF1F73B51F4B01F07F0459
:10FEE00005461B5D83B36FF000720C2100F094FB9C
:10FEF0000E21284600F0B6FB00264FF0FF320C2101
:10FF0000284600F089FB32466D2128460194009670
:10FF1000334600F057FB32466C21284600F07CFB4C
:10FF20000E21284600F09EFB8201F9D56E2128465D
:10FF300000F098FB222C01D0422C03D1030201D502
:10FF400040F07F4002B070BD04EB44040444034B16
:10FF500053F82400F6E700BF6038010034F9FF1FB2
:10FF600070B50B4C2218054692F800260E465AB979
:10FF70006C21FFF7B1FF06F00F0320F00F021A43C8
:10FF80006C212846FFF762FF631983F8036670BD92
:10FF900034F9FF1F38B50C466C210546FFF79CFF6E
:10FFA000240104F0700420F07002224328466C21E2
:10FFB000BDE83840FFF74ABF38B50C466C2105460E
:10FFC000FFF78AFFE40304F4C03420F4C032224374
:10FFD00028466C21BDE83840FFF738BF38B50C46DD
:10FFE0006C210546FFF778FF240504F4700420F423
:10FFF0007002224328466C21BDE83840FFF726BF37
:020000021000EC
:1000000038B50C466C210546FFF766FF240604F060
:10001000706420F07062224328466C21BDE83840AD
:10002000FFF714BF38B50D466C210446FFF754FFA7
:100030003DB140F0804220466C21BDE83840FFF7DA
:1000400005BF20F08042F6E738B50D466C21044626
:10005000FFF742FF3DB140F4002220466C21BDE88D
:100060003840FFF7F3BE20F40022F6E738B50D461E
:100070006C210446FFF730FF3DB140F4802220465A
:100080006C21BDE83840FFF7E1BE20F48022F6E79E
:1000900038B50D466C210446FFF71EFF3DB140F414
:1000A000804220466C21BDE83840FFF7CFBE20F4E7
:1000B0008042F6E738B50D466C210446FFF70CFF89
:1000C0003DB140F4005220466C21BDE83840FFF7B6
:1000D000BDBE20F40052F6E738B50D466C2104464B
:1000E000FFF7FAFE3DB140F4805220466C21BDE896
:1000F0003840FFF7ABBE20F48052F6E738B50C4627
:100100006C210546FFF7E8FE230748BF20F070008A
:100110004FEA04124CBF40F4006020F4076002F084
:10012000700202436C212846BDE83840FFF78EBEBE
:1001300038B50C466C210546FFF7CEFEE40104F409
:10014000F06420F4F062224328466C21BDE8384078
:10015000FFF77CBEFFF7ECBF38B50D466C210446B7
:10016000FFF7BAFE3DB140F4003220466C21BDE8F5
:100170003840FFF76BBE20F40032F6E708B5074BB6
:10018000034493F800262AB96C21FFF7A5FE00F07E
:100190000F0008BD93F8030608BD00BF34F9FF1F28
:1001A00008B56C21FFF798FEC0F3021008BD08B532
:1001B0006C21FFF791FEC0F3C13008BD08B56C217A
:1001C000FFF78AFEC0F3035008BD08B56C21FFF7A6
:1001D00083FEC0F3036008BD08B56C21FFF77CFE09
:1001E000C0F3807008BD08B56C21FFF775FEC0F341
:1001F000C04008BD08B56C21FFF76EFEC0F380401B
:1002000008BD08B56C21FFF767FEC0F3803008BD5C
:1002100008B56C21FFF760FEC0F3403008BD08B59B
:100220006C21FFF759FEC0F3003008BD08B56C2102
:10023000FFF752FEC0F30213020548BF43F0080364
:10024000184608BD08B56C21FFF746FEC0F3C31081
:1002500008BDFFF7F7BF08B56C21FFF73DFEC0F3FF
:10026000404008BD38B50C466D210546FFF734FE09
:10027000640104F0600420F06002224328466D21EE
:10028000BDE83840FFF7E2BD38B50C466D210546A4
:10029000FFF722FE640304F4C04420F4C04222436A
:1002A00028466D21BDE83840FFF7D0BD38B50C4673
:1002B0006D210546FFF710FE240204F4706420F45B
:1002C0007062224328466D21BDE83840FFF7BEBD6D
:1002D00038B50C466D210546FFF7FEFD04F00F040E
:1002E00020F00F02224328466D21BDE83840FFF779
:1002F000ADBD38B50D466D210446FFF7EDFD20F488
:100300007F0040EA05426D212046BDE83840FFF7F6
:100310009DBD38B50D466D210446FFF7DDFD3DB1AD
:1003200040F4004220466D21BDE83840FFF78EBD05
:1003300020F40042F6E738B50D466D210446FFF77C
:10034000CBFD3DB140F0807220466D21BDE83840C4
:10035000FFF77CBD20F08072F6E708B56D21FFF74E
:10036000BBFDC0F3411008BD08B56D21FFF7B4FD1A
:10037000C0F3413008BD08B56D21FFF7ADFDC0F3F6
:10038000032008BD08B56D21FFF7A6FD00F00F00A2
:1003900008BD08B56D21FFF79FFD0314D8B21B06F9
:1003A00048BF60F0FF0008BD08B56D21FFF794FD60
:1003B000C0F3C03008BD08B56D21FFF78DFDC0F357
:1003C000006008BD38B50C4670210546FFF784FD76
:1003D00004F0030420F4401242EA0452284670213B
:1003E000BDE83840FFF732BD38B50D4670210446F0
:1003F000FFF772FD3DB140F4002220467021BDE8B8
:100400003840FFF723BD20F40022F6E738B50D464B
:1004100070210446FFF760FD3DB140F48022204684
:100420007021BDE83840FFF711BD20F48022F6E7C7
:1004300038B50C4670210546FFF74EFD04F0030465
:1004400020F4403242EA044228467021BDE8384098
:10045000FFF7FCBC38B50D4670210446FFF73CFDA4
:1004600020F47F4040EA052270212046BDE8384054
:10047000FFF7ECBC38B50D4670210446FFF72CFDA4
:1004800020F0FF0045EA000270212046BDE8384018
:10049000FFF7DCBC08B57021FFF71EFDC0F301506B
:1004A00008BD08B57021FFF717FDC0F3C04008BDB7
:1004B00008B57021FFF710FDC0F3804008BD08B5F6
:1004C0007021FFF709FDC0F3014008BD08B5702198
:1004D000FFF702FDC0F3072008BD08B57021FFF744
:1004E000FBFCC0B208BD70B50E466C2115461C461B
:1004F00000F0B8F816B1C0F30903336015B1C0F3CA
:1005000004432B700CB1000E207070BD2DE9F34137
:10051000F8F7B4F80446F8F7B1F8001B0028B8BFA4
:1005200040420928F7DD154E0024A046F71EE5B22B
:100530004FF4803200212846FFF788FC0222552321
:100540008DE80C006C21032300222846FFF722FCD3
:100550001F230193009300231A4610212846FFF71A
:1005600019FC2846FFF70AFE04F8078030550134CD
:10057000032CDCD102B0BDE8F08100BF37FFFF1FC4
:1005800038B5074C044494F8001641B994F8035662
:10059000FFF7E6FC012384F8003684F8035638BDE3
:1005A00034F9FF1F064B034493F8002632B10022B2
:1005B00093F8031683F80026FFF7D2BC704700BFFC
:1005C00034F9FF1F2DE9F0411F46124B9DF81860CA
:1005D00033F810409DF81C50904641F080010022F5
:1005E0002046F8F78DFB414600222046F8F788FBAD
:1005F000394600222046F8F783FB31460022204688
:10060000F8F77EFB294620460122BDE8F041F8F7C5
:1006100077BB00BF5480FF1F38B5114B33F8104033
:10062000154641F0800100222046F8F769FB290EAB
:1006300000222046F8F764FBC5F30741002220465C
:10064000F8F75EFBC5F3072100222046F8F758FBB8
:10065000E9B220460122BDE83840F8F751BB00BF9F
:100660005480FF1F38B51E4B33F81040002220463F
:100670000D46F8F745FB002211462046F8F740FBEF
:10068000002211462046F8F73BFB00221146204687
:10069000F8F736FB012200212046F8F731FB294606
:1006A00000222046F8F72CFB002211462046F8F7DE
:1006B00027FB0022114605022046F8F721FB002205
:1006C000114605432046F8F71BFB2D020543012286
:1006D00000212046F8F714FB2D02284338BD00BF47
:1006E0005480FF1F70B504460D461646FFF7BAFF4B
:1006F000294640EA06022046BDE87040FFF78CBF5D
:1007000070B504460D461646FFF7ACFF294620EAB1
:1007100006022046BDE87040FFF77EBF2DE9F84392
:100720009DF8209098460F46064614460025FFF790
:1007300099FFC1444146012349450BD304FA08F40B
:1007400044402C4080EA040239463046BDE8F84374
:10075000FFF762BF03FA01F215430131ECE710B570
:100760000C2104464FF0FF32FFF756FF20460E21C2
:10077000BDE81040FFF776BF10B5CA4304460C2110
:10078000FFF74AFF20460E21BDE81040FFF76ABF81
:1007900010B5084BC4B201221A5420212046002271
:1007A000FFF73AFF204600222421BDE81040FFF762
:1007B00033BF00BFE70300202DE9F7430027714E48
:1007C000714DDFF8CC91B846FCB24FF48052002155
:1007D0002046FFF721FF4FF0051210212046FFF7BA
:1007E0001BFF4A4604212046FFF716FF6FF00072F8
:1007F0000C212046FFF710FF0E212046FFF732FFA5
:1008000000231A466D212046CDF80480CDF80080E3
:10081000FFF7D8FE00226C212046FFF7FDFE0322E1
:1008200005212046FFF7F8FE042220212046FFF78D
:10083000F3FE002237212046FFF7EEFE00222121A1
:100840002046FFF7E9FE4FF4480224212046FFF737
:10085000E3FE4FF4483228212046FFF7DDFE4FF437
:10086000483229212046FFF7D7FEB37D0193737AE2
:10087000B27A0093062100232046FFF7A3FEB38A35
:10088000424A15215A432046FFF7C6FE6A68602196
:100890002046FFF7C1FEAA6861212046FFF7BCFE93
:1008A000EB892A7B1C2143EA02422046FFF7B4FE73
:1008B0002A6959212046FFF7AFFE2A6A5A212046AD
:1008C000FFF7AAFE6A6A5B212046FFF7A5FEAA6A27
:1008D00095F82C30D1B2C2F30722019100925D212C
:1008E00000222046FFF76EFE2A6B5E212046FFF7AE
:1008F00093FEAA6918212046FFF78EFEEA691921A6
:100900002046FFF789FE6A6B5C212046FFF784FED4
:10091000AA6B5F212046FFF77FFEEA6B522120463B
:10092000FFF77AFE6A6C95F84030019395F84130F4
:1009300000936321D3B22046C2F30722FFF742FEA1
:1009400095F84830CDF8048000227D212046CDF86E
:100950000080FFF737FE4FF4403201212046FFF7B9
:100960005BFE01376FF0004235212046FFF754FE51
:10097000032F06F1800605F160057FF425AF03B073
:10098000BDE8F08330040020B405002000710200AF
:100990008D124084034B10229A6000BF00BF00BF3D
:1009A0005A60704700F00F4010B521210446FFF750
:1009B00059FE00F10042013A20463521FFF72CFE96
:1009C0000F212046FFF74EFEC0F3003010BD00029D
:1009D0007047800070470012704780107047704762
:1009E000FEE74FF0E0210B4A0B4BC1F8083D4CF2FB
:1009F0002053D3814DF62813D381138823F00103AC
:100A00001B041B0C1380D1F8883D43F47003C1F81C
:100A1000883D70470020054000800000802800F0DD
:100A20001F014FF001030F4A04DD8B40C2F88C31E7
:100A3000D3607047402804DD8B40C2F88831936052
:100A40007047202804DD8B40C2F884315360704722
:100A5000404200F01F0058BF41428B40C2F8803135
:100A60001360704700E100E0802800F01F024FF0A3
:100A700001030D4903DD9340C1F88C3070474028D5
:100A800003DD9340C1F888307047202803DD934090
:100A9000C1F884307047404200F01F0058BF424206
:100AA0009340C1F88030704700E100E0074B1A78AE
:100AB000D2B2012A02D1222903D15A7001225A70DE
:100AC00070472129FAD10022F7E700BF3AFFFF1F44
:100AD00070B5154611B91B4B197070BD022903D1B1
:100AE000184B01221A7070BD04291AD1154B5B787E
:100AF000012B25D19488402C28BF402400235E1C64
:100B0000DBB2A34207D300231A4602211846BDE8F0
:100B1000704000F047BF2A68D05C00F0C3F833464D
:100B2000EDE7032906D1074A5378012B08D10023AA
:100B30009370E9E7052901BF024B00221A705A7031
:100B400070BD00BF3AFFFF1F10B50446204600F0FD
:100B5000C1F80028FAD110BD704738B50A4C0125FC
:100B600002460B4600202946A57000F0F5FA224601
:100B700018B10023A370122038BD937803F0FF0052
:100B8000002BFAD138BD00BF3AFFFF1FF8B506466B
:100B90000F4600F0F4FC0E4B1A78012A16D15B7850
:100BA000012B13D100F000F988B10025ECB2A74267
:100BB00005D821463046BDE8F840FFF7CEBF3019D2
:100BC00000F0D6F801350028F0D0F2E70C20F8BD8F
:100BD0003AFFFF1F08B540210248FFF7D7FF00F09A
:100BE00095F808BD3DFFFF1F38B5054600F0A8F891
:100BF0000B28044609D140210548FFF7C7FF28B953
:100C00002846BDE8384000F09BB80024204638BD97
:100C10007DFFFF1F70B50C46461E00250CB9284607
:100C200070BD16F8010FFFF7DFFF013C002818BF69
:100C30000B25A4B2F2E738B5451E002415F8010FC4
:100C400008B9204638BDFFF7CFFF002818BF0B2496
:100C5000F4E707B50123002200930649064B10462E
:100C600000F020FA002814BF1B20002003B05DF81C
:100C700004FB00BFD10A0100AD0A010038B50C46E3
:100C8000054600F097F8A0420AD32C440020A54264
:100C900007D000B138BD15F8010B00F051F8F6E7A8
:100CA0000B2038BD10B50A4A117840290ED0537870
:100CB000D4180133DBB2402BA07001F101014FF0D9
:100CC0000000117014BF5370507010BD0B2010BD88
:100CD000BDFFFF1F10B50C4A117891B192F8423058
:100CE000D4180133DBB2A4780470402B4FF000001D
:100CF00001F1FF31117014BF82F8423082F84200D6
:100D000010BD0A2010BD00BFBDFFFF1F014B1878AA
:100D1000704700BFBDFFFF1F024B1878C0F14000B5
:100D2000C0B27047BDFFFF1F034B00225A7083F80B
:100D300042201A70704700BFBDFFFF1FFFF7F4BFCE
:100D400010B50A4A117840290ED05378D4180133CF
:100D5000DBB2402BA07001F101014FF000001170D7
:100D600014BF5370507010BD0B2010BD0000002048
:100D700010B50C4A117891B192F84230D418013371
:100D8000DBB2A4780470402B4FF0000001F1FF317A
:100D9000117014BF82F8423082F8420010BD0A2060
:100DA00010BD00BF00000020014B1878704700BF45
:100DB00000000020024B1878C0F14000C0B270471C
:100DC00000000020034B00225A7083F842201A7062
:100DD000704700BF00000020FFF7F4BF70B5054664
:100DE000007801F093F902780023D9B2914207D23A
:100DF0005C1C03EB830303445E786B789E4227D12F
:100E0000174C2B7A342202FB0142D67813B33423D9
:100E10004B43E218907886420CD000F00302043372
:100E20000C2010FB02302118205C0B894A6849789D
:100E300000F090FBD4F89C3083B12A46287812F851
:100E4000081F00290CBF03210521BDE87040184789
:100E50002346CAE7937801339370D8E770BD00BF8B
:100E6000440000202DE9F04F85B00D4690468DF8E6
:100E70000F0001F04BF9022D064647D107780023F9
:100E80005C1CDBB2BB4210DB4FF00009DFF8B0B0F6
:100E9000CA465FFA89F4A74212DC284BD3F89C308B
:100EA000002B45D105B0BDE8F08F03EB830333443D
:100EB0000DF10F00DA78597801F0E2F92346DFE707
:100EC00004EB84043444E378A2886178CDF804A06C
:100ED000A07800900DF10F0001F0B0F9A378032B7A
:100EE00005D15A4661789DF80F0001F031FA61781A
:100EF000E37841F0100141EAC3110022C9B20DF1BB
:100F00000F0001F0EDF909F10109C2E7002DC4D18C
:100F10000A490378342000FB03138A1C3633294620
:100F200034329A42B9D002F8341C02F8331CF7E785
:100F3000424629469DF80F009847B3E74400002039
:100F4000DD0D0100F0B40C7804F06004202C1D4687
:100F500032D14C78042C1DD00AD8012C04D003D3F4
:100F6000022C20D0032C12D000202880F0BC704727
:100F7000212C1BD004D8202CF6D1F0BC00F040B9B5
:100F8000222C16D0232CEFD1F0BC00F049B9F0BCD4
:100F900000F049B902241C801468002525701468EB
:100FA000671C17606570F0BC00F056B9F0BC00F02B
:100FB0001FB9F0BC00F076B9402C06D1044CD4F82F
:100FC000A04014B1A446F0BC6047CD20CEE700BFDE
:100FD0004400002073B50446007801F097F8636878
:100FE0000093A27A637A43EA0223ADF804300278D0
:100FF0000023D9B2914207D25D1C03EB8303034463
:101000005E7863789E4225D1174D237A342202FB05
:101010000152D67803B334234B43EA1890788642C2
:101020000CD000F0030204330C2010FB023029180E
:10103000285C0B894A68497800F08CFAD5F89C3016
:1010400033B1227A20785AB104F108020521984779
:1010500002B070BD2B46CCE7937801339370DAE78A
:101060006A460321F3E700BF4400002007B5436848
:101070000093437A817A43EA0123ADF80430084BA8
:10108000D3F89C3002462BB1017A007829B108329E
:101090000521984703B05DF804FB6A460421F8E790
:1010A000440000202DE9F84305460F4616469846B1
:1010B00001F02CF802789DF8203001328146D2B23E
:1010C0000021284601F09EF80446E8B9164A17495F
:1010D000284600F086F999F80000154B342200FBF1
:1010E000022209F101011A4499463433934201F175
:1010F00005010CD14146284600F074F8044618B9A1
:10110000C9F89C70C9F8A0602046BDE8F88311F8C2
:10111000050C03F8340C11F8040C03F8330C03F835
:10112000324C03F8314CE0E7450F0100650E010039
:101130004400002008B5074B0022C3F89C20C3F8E8
:10114000A02000F0A1F918B9BDE8084001F06EB880
:1011500008BD00BF440000202DE9F0419846054637
:101160000E46174600F0D2FF04780023D9B2A14200
:1011700007D2013303EB8302024412F8042CB2427B
:10118000F4D1174C34234B43E218D07892F802E0A4
:10119000A0EB0E01C9B2042902D1C120BDE8F08143
:1011A00000F003010130C0B24FF00C0C0CFB013316
:1011B000D070A0EB0E001C44C0B2012825716671EE
:1011C000A760A4F80C8007D143463A46314628462A
:1011D000BDE8F04100F0BEB90020BDE8F08100BFDD
:1011E00044000020014B002019607047E8000020F7
:1011F000024B0979197100F08DBF00BFE800002093
:1012000013B5002402AA1C80044B42F8041D09797E
:10121000197100F08DFF02B010BD00BFE800002082
:1012200000201880704730B40C46022119802179C3
:101230006488084D012C297102D130BC00F08EBFAA
:10124000022C02D130BC00F095BF0020188030BCC9
:10125000704700BFE800002030B40C46022119801E
:1012600021796488074D012C297102D130BC00F02E
:101270008DBF022C02D130BC00F09ABF0020188034
:1012800030BC7047E8000020044B054A19795B79AF
:101290001171137203210A23FFF75EBFE8000020DB
:1012A0005A80FF1FF8B500271F808B780B4CA37165
:1012B000C3F340035A0063F3000206466271FFF76E
:1012C000E3FF256845B1A37913F002021ABF3A463D
:1012D000222121213046A8470020F8BDE800002047
:1012E000034B00F108021B6800780521184700BF76
:1012F000F000002070B5094D04462A1D012100F0C0
:10130000D7FF80220121204600F0EAFF2B682078D9
:1013100000220A21BDE87040184700BFF0000020FD
:1013200037B501210DF10702044600F0C1FF9DF819
:101330000730074D802B04D12A790121204600F087
:10134000CFFF2B68207800220B21984703B030BDD7
:10135000F0000020436805215A7800F0C1BF73B542
:101360000122002405460126002100F089FF3346B2
:1013700021468DE850001022284600F05FFF2246EB
:101380002146284600F07CFF234621468DE8500088
:101390001022284600F052FF31460222284600F073
:1013A0009FFF32460621284600F09AFF22469021F0
:1013B000284600F095FF044B28781B6822462146FA
:1013C00002B0BDE870401847F000002042783AB9FA
:1013D000C178C90141F0100101F0900100F080BF17
:1013E000704773B50C468DF8070001F00DFA1F4DDC
:1013F0002C600446002836D11D4A9DF807001021B4
:1014000000F0A6FF1B4A044612219DF8070000F0D9
:101410009FFF194A044314219DF8070000F098FF2C
:10142000E4B20443154A9DF80700132100F090FF31
:10143000E4B20443124A9DF80700172100F088FF28
:1014400002AEE4B204430F4A16F8010D162100F073
:101450007FFFE4B2044303220121304600F040FF45
:101460000323E4B22B71204602B070BDF0000020CF
:101470005F13010055130100F51201002113010053
:10148000CD130100E112010037B502AD174B05F88D
:10149000010D0022102128461A6000F05BFF122186
:1014A0000446284600F056FF14210443284600F065
:1014B00051FFE4B204431321284600F04BFFE4B28D
:1014C00004431721284600F045FFE4B204431621E7
:1014D000284600F03FFFE4B2204310F0FF0003D1A4
:1014E0009DF8070001F09CF903B030BDF00000202A
:1014F0001FB501218DF807000DF10E020DF1070057
:1015000000F0D6FE0DF10F0206210DF1070000F0EC
:10151000CFFE9DF80E30802B18D19DF80F309B0721
:1015200014D59DF8070000F0EFFD012804460DD109
:1015300072B60DF1070000F029FB002221460DF1E3
:1015400007008DF80E2000F0CBFE62B69DF80E006D
:1015500004B010BD73B50C4615461E468DF8070045
:10156000FFF7C6FF802808D033462A4621460DF1F2
:10157000070000F0A7FA02B070BD0020FBE770473B
:10158000062812D880000129C0B201D10230C0B2B1
:10159000074AC0F34703122101FB03231A884FF6C1
:1015A000FF739A4208BFFF207047FF20704700BFBB
:1015B000F80000202DE9F041314C324D324E4FF011
:1015C000000884F800814FF4107285F840020F463D
:1015D0002846FF2101F0DEFF4FF48062414630468D
:1015E000C5F8446201F0D6FF94F80C3143F0800353
:1015F00084F80C3194F80C311B06FBD4234BFF22EA
:101600001A7094F80C3143F0400384F80C31204BED
:10161000196897B341F000411960194B310AC6F3BC
:10162000074201F0FE0183F89C1083F8B020320ECF
:1016300083F8B420174AC5F84822102283F80821FD
:10164000012283F89420BF2283F8802093F80021A0
:1016500002F07F0283F8002193F8842042F0010217
:1016600083F8842093F8842042F0100283F88420C9
:1016700084221A770020BDE8F08121F00041CBE7F9
:1016800000200740F8000020000E00206480FF1FAB
:1016900000700440001000200D4B93F80C2102F064
:1016A000BF0283F80C21BF2283F8802093F88420A6
:1016B00002F0FE0283F8842093F8942002F0FE02E8
:1016C00083F894201A7F02F07B021A77002070477B
:1016D00000200740F7B5082304248DE81800B1F86E
:1016E00003300D788878B3F5007F81BF0023CB707D
:1016F00002230B71062D71D8AB00DCB2012804BFA8
:101700000234E4B24FEA540E354C122707FB0E4761
:101710004FF6FF76B7F800C0B4455FD14E78032E80
:101720005CD801285AD897F80FC0BCF1FF0F04BF4E
:101730004FF0000C87F80FC0B1F803C0122101FB75
:101740000EFE04EB0E0743EA4003BA73FA7B7E7485
:1017500002F0010213435BB2D4F84822C7F802201A
:10176000D9B2F9733874D4F8447224F80EC01BB29D
:1017700007EBC30E81F00101CEF80420AEF802C0E1
:101780004FF0080E07F833E007EBC10ECEF8042047
:10179000AEF802C012FA8CF24FF0480E07F831E0B2
:1017A000C4F8482228B917F8332062F07F0207F8FE
:1017B000332002AA02EB80002DB20A4950F8082C0F
:1017C00011F82530012E0CBF164642F001063343B6
:1017D000DBB201F82530002003B0F0BD9520FBE717
:1017E000F8000020C0200740084610B51146FFF75A
:1017F000C7FEFF281DD0104B1221C0F3470001FB8C
:101800000030D3F84422C37B1CB283F0010312F8EA
:10181000341001F07F0102F8341012F8331001F097
:101820007F0102F833104FF0FF338372C372002040
:1018300010BDC42010BD00BFF800002073B50C46D9
:101840008DF80700114620461646FFF799FEFF283F
:10185000054620D0214632460DF10700FFF7C4FFB0
:10186000C5F3470312210D4D59436B18D5F8482293
:101870001888121AC5F8482224B2094A002002F832
:1018800024004FF0FF326A549A705A70DA701A715D
:101890005A7102B070BD9620FBE700BFF80000202F
:1018A000C02007402DE9F0410E46804611463046E3
:1018B0001746FFF765FE0C4DC0F34700122303FBEC
:1018C0000050C47BFF2C0DD03A4631464046FFF70E
:1018D0008BFF24B2D5F8442212F8343063F07B0336
:1018E00002F83430BDE8F081F800002010B5084659
:1018F00000211446FFF744FE084AC0F347001221B6
:1019000001FB0020D2F84432C27B03EBC2035A68C9
:10191000136823605368636010BD00BFF8000020A7
:1019200010B50C4620461146FFF72AFEFF281AD0B4
:1019300024B2104B13F82430DBB213F00C0F12D08A
:101940009B0712D40C4BD3F8443213F83020D20941
:101950000DD180F00100C0B213F83030DB0914BFA4
:101960000320002010BD052010BD012010BD032064
:1019700010BD00BFC0200740F800002008B5FFF7E9
:10198000FFFD074A1223C0F3470003FB0020C37B7F
:10199000FF2B1EBFD2F84422002102F8331008BDED
:1019A000F80000202DE9F0410846002190461F462E
:1019B000FFF7E6FD2249C0F34700122404FB0014A0
:1019C000E57BFF2D39D022884FF6FF7093B283421A
:1019D00033D0D1F8441285F0010011F9300000280D
:1019E0002BDB2EB287B901EBC60338465A80D4F8F8
:1019F00002205A6011F8352002F0400262F07702AE
:101A000001F83620BDE8F08101EBC602BB424FF081
:101A1000000028BF3B466781C4F8068020736073CE
:101A20005380C2F8048011F8353003F0400363F0AE
:101A3000770301F83630BDE8F0819420BDE8F081ED
:101A4000F80000202DE9F0410C46064611462046DC
:101A50001546FFF795FD194BC0F34700122202FB14
:101A6000003090F80FE0BEF1FF0F24D027B2144AE7
:101A70006CB1407C012D0CBF14211821012818BF26
:101A800041F0010112F82700014302F8271012F873
:101A900027106FF3410102F82710D3F844320022D7
:101AA00003F83E203DB92B462A4621463046BDE884
:101AB000F041FFF777BFBDE8F08100BFF8000020DC
:101AC000C02007402DE9F0410C4620460121174671
:101AD0009846FFF755FDFF2836D01C4BC0F3470052
:101AE000122202FB0030D3F8446290F80FE016F99E
:101AF0003E30002B28DB23B2154A12F8235015F094
:101B0000020521D10188C0F806701FFA88F24281CF
:101B10008A42D8BF11460FFA8EF206EBC203057354
:101B2000457359805F602CB9C82306F832302046CF
:101B3000BDE8F08116F83E3003F0400363F0770310
:101B400006F832302C46F2E79324F0E7F800002044
:101B5000C0200740034B044883F898100122114627
:101B600000F0BEBB0020074038030020054B0648AC
:101B7000002283F89420802283F80C210121FF2287
:101B800000F0AEBB002007403803002038B51A4CE7
:101B900094F8002102F07F0284F8002194F80C21CF
:101BA00002F0DF0284F80C2194F8802042F0200239
:101BB00084F8802094F8842002F0DF0284F88420E6
:101BC00094F8942002F0DF0284F8942094F8942092
:101BD00042F0040284F8942044F62065013DADB241
:101BE00000F0BCFE002DF9D194F8943003F0FB0313
:101BF00084F8943038BD00BF002007402DE9F04F35
:101C0000D84DD94C95F8807095F8843095F890604F
:101C100087B0FF221F4094F840328DF809208DF8DC
:101C20000C308DF80D20002301210DF1090204F57F
:101C300010708DF80E3004938DF815308DF8163035
:101C40008DF80F308DF8143000F032FB95F80C3120
:101C5000D907F6B20FD59DF80930802B0BD195F836
:101C6000003103F07F0385F8003195F80C3103F063
:101C7000DF0385F80C317A0711D5BA4B042093F8AD
:101C8000A41093F8A02083F8800006AB42EA01225A
:101C900023F80E2D03A91220049300F06DFBFB071F
:101CA0004BD5B04DB0480123BF2685F8803085F86C
:101CB000886095F89430002743F0020385F894304B
:101CC0004FF4107285F89870FF2185F8007101F0CB
:101CD00061FC4FF480623946D4F8440201F05AFCAA
:101CE000D4F8443203F50073C4F848329F4BFF2206
:101CF0001A7095F8943003F0FD0385F8943095F848
:101D00000C3143F0400385F80C319F2385F88C603B
:101D100085F8843095F8943003F0DF0385F894302B
:101D200003A9102000F028FB95F8943003F0DF039E
:101D300085F8943007B0BDE8F08F3D0740F19380FF
:101D4000884B082283F880203309C6F3C000062B95
:101D50008DF80D308DF80F0000F2F480C6F380028C
:101D600002EB830208B10232D2B2D4F8446206EB2D
:101D7000C201C2F34705D1F804E04988ADF8151057
:101D8000122101FB0541CDF810E091F80FC08CF055
:101D9000010C81F80FC016F8321082F0010A5FFAC8
:101DA0008AFAC1F380110FFA8AF881F001018901E2
:101DB00006EBC80906F83810002800F0D980DFF8D3
:101DC000ACB19BB99BF8002082B9FF2219468BF871
:101DD000002003A81A460193FFF706FD019B06F8B1
:101DE00038301A46194603A8FFF7DCFD9BF800308F
:101DF000012B04D09DF80D30002B00F0AD80122196
:101E000001FB0541BDF815008B894A8903449BB24B
:101E100093428B8109D3B1F800E0C0B2864540F00F
:101E20009380897B012940F08F80122101FB0544BA
:101E3000D4F8061020881944D31A8342D8BF98B228
:101E4000A9F80200C9F8041016F83A3003F040036C
:101E500063F0770306F83830424A92F8943003F082
:101E6000DF0382F89430B80717D53E4C022384F87C
:101E7000803094F8883094F88C2003A91340162001
:101E80008DF8143000F078FABF2384F8883094F885
:101E9000943003F0DF0384F89430F9061CD5314CFC
:101EA000202384F88030102384F8803003A9142084
:101EB00000F062FA94F80C3143F0200384F80C31FE
:101EC00094F8003143F0800384F8003194F88430B2
:101ED00043F0200384F88430BA060DD5214C20232A
:101EE00084F8803003A9132000F046FA94F8843077
:101EF00003F0DF0384F884303B067FF51BAF0DF160
:101F00000A02FF23102103A88DF80D3000F0D0F94C
:101F10009DF80A30134C012B04BF8DF80F300022BE
:101F20004FF0800308BF8DF80D2003A984F880309E
:101F3000172000F021FA94F8943003F0DF0384F8BE
:101F40009430F7E6FF2210E7122202FB0544D4F892
:101F500006200492ADF8153003A99DF80D0000F09D
:101F60000BFA79E700200740F80000206480FF1F8B
:101F70006BB916F832202F4902F03C02342A35D1D1
:101F800001238DF80E309EF80030DB090B70122112
:101F900001FB05414FF6FF734A899A42DCD0BDF838
:101FA00015E08B8973449BB28B8109888E4501D1E2
:101FB0009A420CD88AB3B2FBF1F001FB102080B238
:101FC00058BB122000FB0540807B012825D1D21A86
:101FD0008A42D8BF91B2122202FB0544C9B9D4F893
:101FE0000230C9F80430A9F802102DE70A78012A56
:101FF000CDD1FF200870194603A80193FFF7F4FB29
:10200000019B06F838301A46194603A8FFF7CAFCA8
:10201000BDE7D4F806201344E3E7122202FB05448F
:10202000D4F80620ADF815304FF0FF330492A372B8
:10203000E37291E76480FF1F13460A46194601F0D8
:10204000A9BA00BF30B50329039C04981DD12BB950
:10205000164A226004220280002030BD40F209416D
:102060008B420FD1022A4FF000030CD810490C25E7
:1020700005FB0313D9681B6951F8221021609B5C92
:102080000380E9E701230122F0E7072901D9CD20E8
:1020900030BD074B03EB8102126A2260002AF6D0A2
:1020A00003EB4103B3F84030EAE700BF6580FF1F50
:1020B000E038010001299FBF034B5B5C13700020D7
:1020C00088BFCD20704700BF4403002001299DBF79
:1020D000024B00205A54CD20704700BF440300201B
:1020E00019B14B1E58425841704701207047054BAB
:1020F0001A788A4204D05878431A58425841704797
:1021000001207047440300200020704700487047BA
:102110003039010001299FBF044BC1EBC101C9182F
:10212000002094BF1160CD20704700BF6980FF1F61
:10213000012930B50ED8084DC1EBC1010823106844
:10214000C45CC818284401330F2B00F8084CF6D1A2
:10215000002030BDCD2030BD6980FF1F01299FBF09
:10216000034B03EB41010020116088BFCD20704775
:102170004603002001299FBF034B03EB41010020D0
:10218000116088BFCD2070474A03002001290AD87A
:1021900013681878054B03EB4101887013685B786E
:1021A000CB7000207047CD20704700BF4403002053
:1021B00001290AD813681878054B03EB410188718F
:1021C00013685B78CB7100207047CD20704700BF4B
:1021D00044030020084B5A7803F8022BFF21002209
:1021E000D1540132072AFBD1044A00230521995416
:1021F0000133072BFBD170474E030020570300200B
:1022000000BF7047013AD2B2062A10B51C4608D862
:10221000054B5A70FFF7DEFF2146BDE81040FFF77F
:10222000C9B9992010BD00BF4E030020024B002207
:102230005A70FFF731BA00BF4E03002037B50F4C7C
:10224000257805B9C1B98DF802308DF800109DF8D8
:102250001830ADF8032069469DF81C2000788DF8F1
:102260000130FFF737FA9DF800301BB110B9237821
:10227000013B237003B030BD9520FBE74E030020E7
:1022800038B50A4B0D461C7859788C421C4600D153
:102290004DB929460078FFF7D1FA2DB120B923783E
:1022A0000133237038BD962038BD00BF4E03002097
:1022B0004B1E062B05D8094B19444B781370002090
:1022C0007047CB0607D501F00F01062903D8034B51
:1022D00019444B7AF2E78220704700BF4E0300207A
:1022E0004B1E062B2DE9F0418046174605D8174BAB
:1022F00019444A700020BDE8F081CB0622D501F0D8
:102300000F05062D1ED8012A4FEAD1140F4E06D113
:1023100022462946FFF7C6FA35446F72EAE7002ADB
:10232000FAD173195B7A012BF6D122462946FFF7C1
:1023300089FB002DF0D184F0010229464046FFF7C9
:1023400081FBE9E78220BDE8F08100BF4E03002059
:1023500000207047062903D9A1F11003072B07D8E5
:10236000044B53F82130002B0CBFC42000207047D1
:10237000C420704758390100102810B50C4601D10F
:10238000FFF728FF034B53F820300BB12046984746
:10239000002010BD583901001FB5144602228DF8E7
:1023A00007001A8005210DF10F020DF10700FFF75C
:1023B0007FFF034B9DF80F201A80236004B010BDEF
:1023C000600300201FB5144601228DF807001A8013
:1023D00004210DF10F020DF10700FFF769FF044B17
:1023E0009DF80F201A800020236004B010BD00BFAC
:1023F00060030020F0B5002685B01E8049888DF866
:102400000700ADF80E10FFF76BFE18B3BDF80E20F5
:10241000114F04ACB2FA82F2520901210DF107000A
:10242000FFF75EFF34F8022D0421D2B20DF1070050
:10243000FFF756FF7B682246012105469DF80700FD
:1024400098477B689DF80700324602219847284646
:1024500005B0F0BD0425FAE76003002073B502ACB7
:10246000002504F8010D0E461D800422012120469E
:10247000FFF736FF7288024B28461A7202B070BD11
:102480006003002013B54C8889888DE80C000B464A
:10249000E2B2210AFFF7D6FD02B010BD2DE9F041EE
:1024A00086B017461E4606AA0023884605930323D6
:1024B0008DF80F0002F8083D01210DF10F00FFF724
:1024C000F7FE98F80050274C15F0030528D10DF1C0
:1024D000110206210DF10F00FFF7EAFE9DF8113001
:1024E0009DF80F0003F0030323800DF11203019305
:1024F00005AB00932A462B460221FFF7A3FD059B5F
:10250000DB7913F0400F238814BF43F0010323F05D
:1025100001032380022333803C6006B0BDE8F081D4
:10252000012D08D19DF81030012B02D198F804300C
:10253000ABB90023EDE7022DEED198F8041041F07D
:1025400010010DF11202C9B20DF10F00FFF7B0FE3C
:102550009DF8123003F0010323803580DCE7CD20A5
:10256000DAE700BF600300207FB500221A800B78F5
:102570004E788DF8070013F003030D46C6F34006AE
:1025800034D1FEB14B88013B9BB2012B52D80DF1E7
:102590000F0206210DF10700FFF78AFE044670B90D
:1025A000AB7801229A409DF80F301A43D2B206212F
:1025B0000DF107008DF80F20FFF792FE044620462C
:1025C00004B070BD4E88012E34D10DF10F020621EA
:1025D0000DF10700FFF76CFE04460028EFD1AA7842
:1025E00096409DF80F2022EA0602E0E7022B21D157
:1025F00009798DF80F10324641F010010DF10700F6
:10260000FFF76EFE6B78002E14BF07210821012B07
:10261000044607D19DF80F00C10900F00F00FFF735
:10262000ADF90821044B9DF807005B680DF10F021E
:102630009847C4E7CD24C2E76003002010B500240A
:102640001C800B7803F00303012B05D18A780979EC
:10265000FFF73CFD204610BD042010BD38B51546DF
:102660000A7802F00302012A07D1054C1A80097981
:102670002246FFF71FFD2C6038BD042038BD00BF87
:102680006003002013B5CD298DF8070007D1012282
:1026900090210DF10700FFF723FE02B010BD0D4998
:1026A0001C88088A1268844288BF18800C461B88E0
:1026B0009DF807000021FEF74DFF94F90A30002B2A
:1026C000EBDA00231A4619460DF10700FFF76AF905
:1026D000E3E700BF6003002073B5054600266A46A5
:1026E00001218DF800600196FFF7E2FDAA78434CC6
:1026F000012A52D168680368C4F80A304368A07A96
:10270000C4F80E3004F10A0110F0600F1ED1E27A15
:102710003B4B53F82240002C3DD09DF8000002288E
:1027200039D802EB42021344034493F83430012BAE
:1027300031D10DF1020301AA2878A0470DF102035F
:1027400001AA01462878FFF79DFF13E0238AADF820
:102750000230202B17D87BB102060DD40A68C4F8CA
:1027600012204A68C4F81620314604F11A0228469D
:10277000FFF718F902B070BDE46B64B10DF102030C
:1027800001AA2049D8E702A82B7800F8073D90213C
:10279000FFF7A6FDEEE7CD20D0E79DF80030042B33
:1027A00010D12B78217A02AD05F8063D2846FFF7B7
:1027B000D1F9012211462846FFF792FD227A032122
:1027C0002846E5E794F90A30002BD3DBEB78002BA1
:1027D000D0D1E66B86B1B5F8093028780833ADF86A
:1027E000023004F112010DF1020301AAB0470146C3
:1027F0000DF1020301AAA5E7CD21F9E7600300204E
:10280000B83901006A030020034B5960DA630021E4
:10281000024AFFF79DBD00BF60030020D9260100DA
:1028200007B502AB054A03F8010D002118465160B7
:10283000D163FFF78FFD03B05DF804FB6003002058
:1028400000207047354B41F248015A5822F00F02E0
:1028500042F002025A5041F204015A5842F48022D6
:102860005A5041F234015A5842F480225A5003F52A
:102870002C33602193F8942042F0020283F89420D4
:10288000C02283F80021FF221A7483F8802083F885
:10289000882083F88420002283F88C2083F80C1190
:1028A0001F491A75080A00F0FE0083F8982083F883
:1028B000C02083F8C42083F8C82083F8CC2083F894
:1028C000D02083F8D42083F8D82083F8DC2083F844
:1028D000E02083F8E42083F8E82083F8EC2083F8F4
:1028E000F02083F8F42083F8F82083F8FC2083F8A4
:1028F0009C00C1F30740090E83F8B00083F8B410C0
:1029000083F8AC201A7783F8082193F8942002F01A
:10291000D40242F0010283F8942070470070044012
:10292000000E0020024B4FF400125A60704700BFA7
:1029300000E100E0034B4FF40012C3F884215A6019
:10294000704700BF00E100E008B5FEF782F910B95A
:10295000FFF7F0FF08BD1B2008BD00BF034B4AF284
:1029600002629A814BF280429A81704700200540B2
:10297000844641EA000313F003036DD1403A41D38A
:1029800051F8043B40F8043B51F8043B40F8043B49
:1029900051F8043B40F8043B51F8043B40F8043B39
:1029A00051F8043B40F8043B51F8043B40F8043B29
:1029B00051F8043B40F8043B51F8043B40F8043B19
:1029C00051F8043B40F8043B51F8043B40F8043B09
:1029D00051F8043B40F8043B51F8043B40F8043BF9
:1029E00051F8043B40F8043B51F8043B40F8043BE9
:1029F00051F8043B40F8043B51F8043B40F8043BD9
:102A0000403ABDD2303211D351F8043B40F8043B78
:102A100051F8043B40F8043B51F8043B40F8043BB8
:102A200051F8043B40F8043B103AEDD20C3205D388
:102A300051F8043B40F8043B043AF9D2043208D080
:102A4000D2071CBF11F8013B00F8013B01D30B88F2
:102A500003806046704700BF082A13D38B078DD0D0
:102A600010F003038AD0C3F10403D21ADB071CBFA2
:102A700011F8013B00F8013B80D331F8023B20F80C
:102A8000023B7BE7043AD9D3013A11F8013B00F845
:102A9000013BF9D20B7803704B7843708B788370CD
:102AA0006046704781F0004102E000BF83F00043C0
:102AB00030B54FEA41044FEA430594EA050F08BFD9
:102AC00090EA020F1FBF54EA000C55EA020C7FEA9D
:102AD000645C7FEA655C00F0E2804FEA5454D4EB1A
:102AE0005555B8BF6D420CDD2C4480EA020281EAE4
:102AF000030382EA000083EA010180EA020281EA1C
:102B00000303362D88BF30BD11F0004F4FEA01316D
:102B10004FF4801C4CEA113102D0404261EB41017C
:102B200013F0004F4FEA03334CEA133302D0524202
:102B300063EB430394EA050F00F0A780A4F10104BE
:102B4000D5F1200E0DDB02FA0EFC22FA05F28018F8
:102B500041F1000103FA0EF2801843FA05F35941DE
:102B60000EE0A5F120050EF1200E012A03FA0EFC5D
:102B700028BF4CF0020C43FA05F3C01851EBE37187
:102B800001F0004507D54FF0000EDCF1000C7EEBA4
:102B900000006EEB0101B1F5801F1BD3B1F5001FE2
:102BA0000CD349085FEA30004FEA3C0C04F1010401
:102BB0004FEA445212F5800F80F09A80BCF1004F2A
:102BC00008BF5FEA500C50F1000041EB045141EAAC
:102BD000050130BD5FEA4C0C404141EB010111F4AD
:102BE000801FA4F10104E9D191F0000F04BF014658
:102BF0000020B1FA81F308BF2033A3F10B03B3F136
:102C000020020CDA0C3208DD02F1140CC2F10C02C5
:102C100001FA0CF021FA02F10CE002F11402D8BF23
:102C2000C2F1200C01FA02F120FA0CFCDCBF41EAEF
:102C30000C019040E41AA2BF01EB0451294330BDBE
:102C40006FEA04041F3C1CDA0C340EDC04F114049B
:102C5000C4F1200220FA04F001FA02F340EA030072
:102C600021FA04F345EA030130BDC4F10C04C4F1B8
:102C7000200220FA02F001FA04F340EA0300294698
:102C800030BD21FA04F0294630BD94F0000F83F4E2
:102C9000801306BF81F480110134013D4EE77FEAC5
:102CA000645C18BF7FEA655C29D094EA050F08BF11
:102CB00090EA020F05D054EA000C04BF19461046F2
:102CC00030BD91EA030F1EBF0021002030BD5FEA36
:102CD000545C05D14000494128BF41F0004130BD5E
:102CE00014F580043CBF01F5801130BD01F00045B2
:102CF00045F0FE4141F470014FF0000030BD7FEA25
:102D0000645C1ABF194610467FEA655C1CBF0B461F
:102D1000024650EA013406BF52EA033591EA030F36
:102D200041F4002130BD00BF90F0000F04BF00212E
:102D3000704730B54FF4806404F132044FF0000561
:102D40004FF0000150E700BF90F0000F04BF0021DA
:102D5000704730B54FF4806404F1320410F0004540
:102D600048BF40424FF000013EE700BF42004FEA3B
:102D7000E2014FEA31014FEA02701FBF12F07F43B8
:102D800093F07F4F81F06051704792F0000F14BFB5
:102D900093F07F4F704730B54FF4607401F00045F9
:102DA00021F0004120E700BF50EA010208BF704750
:102DB00030B54FF000050AE050EA010208BF704745
:102DC00030B511F0004502D5404261EB41014FF4AE
:102DD000806404F132045FEA915C3FF4DCAE4FF0B2
:102DE00003025FEADC0C18BF03325FEADC0C18BF99
:102DF000033202EBDC02C2F1200300FA03FC20FAEA
:102E000002F001FA03FE40EA0E0021FA02F1144436
:102E1000C1E600BF70B54FF0FF0C4CF4E06C1CEA4B
:102E200011541DBF1CEA135594EA0C0F95EA0C0FC0
:102E300000F0DEF82C4481EA030621EA4C5123EA33
:102E40004C5350EA013518BF52EA033541F4801162
:102E500043F4801338D0A0FB02CE4FF00005E1FB15
:102E600002E506F00042E0FB03E54FF00006E1FB5F
:102E700003569CF0000F18BF4EF0010EA4F1FF04A2
:102E8000B6F5007F64F5407404D25FEA4E0E6D41E2
:102E900046EB060642EAC62141EA55514FEAC520F3
:102EA00040EA5E504FEACE2EB4F1FD0C88BFBCF56F
:102EB000E06F1ED8BEF1004F08BF5FEA500E50F120
:102EC000000041EB045170BD06F0004646EA0101E6
:102ED00040EA020081EA0301B4EB5C04C2BFD4EB18
:102EE0000C0541EA045170BD41F480114FF0000E11
:102EF000013C00F3AB8014F1360FDEBF002001F07F
:102F0000004170BDC4F10004203C35DA0C341BDCF8
:102F100004F11404C4F1200500FA05F320FA04F0CA
:102F200001FA05F240EA020001F0004221F00041FE
:102F300010EBD37021FA04F642EB06015EEA430E71
:102F400008BF20EAD37070BDC4F10C04C4F12005A1
:102F500000FA04F320FA05F001FA04F240EA020054
:102F600001F0004110EBD37041F100015EEA430E25
:102F700008BF20EAD37070BDC4F1200500FA05F245
:102F80004EEA020E20FA04F301FA05F243EA0203C4
:102F900021FA04F001F0004121FA04F220EA0200D3
:102FA00000EBD3705EEA430E08BF20EAD37070BD19
:102FB00094F0000F0FD101F00046400041EB0101F9
:102FC00011F4801F08BF013CF7D041EA060195F0DB
:102FD000000F18BF704703F00046520043EB030395
:102FE00013F4801F08BF013DF7D043EA0603704782
:102FF00094EA0C0F0CEA135518BF95EA0C0F0CD08D
:1030000050EA410618BF52EA4306D1D181EA0301D2
:1030100001F000414FF0000070BD50EA410606BFCC
:103020001046194652EA430619D094EA0C0F02D111
:1030300050EA013613D195EA0C0F05D152EA033656
:103040001CBF104619460AD181EA030101F0004174
:1030500041F0FE4141F470014FF0000070BD41F0BD
:10306000FE4141F4780170BD70B54FF0FF0C4CF497
:10307000E06C1CEA11541DBF1CEA135594EA0C0FB6
:1030800095EA0C0F00F0A7F8A4EB050481EA030E03
:1030900052EA03354FEA013100F088804FEA0333EA
:1030A0004FF0805545EA131343EA12634FEA0222B8
:1030B00045EA111545EA10654FEA00260EF0004179
:1030C0009D4208BF964244F1FD0404F5407402D2CB
:1030D0005B084FEA3202B61A65EB03055B084FEA5C
:1030E00032024FF480104FF4002CB6EB020E75EB59
:1030F000030E22BFB61A754640EA0C005B084FEA81
:103100003202B6EB020E75EB030E22BFB61A7546FD
:1031100040EA5C005B084FEA3202B6EB020E75EB48
:10312000030E22BFB61A754640EA9C005B084FEAC0
:103130003202B6EB020E75EB030E22BFB61A7546CD
:1031400040EADC0055EA060E18D04FEA051545EABC
:1031500016754FEA06164FEAC30343EA52734FEA65
:10316000C2025FEA1C1CC0D111F4801F0BD141EADE
:1031700000014FF000004FF0004CB6E711F4801F43
:1031800004BF01430020B4F1FD0C88BFBCF5E06F23
:103190003FF6AFAEB5EB030C04BFB6EB020C5FEA33
:1031A000500C50F1000041EB045170BD0EF0004E88
:1031B0004EEA113114EB5C04C2BFD4EB0C0541EABA
:1031C000045170BD41F480114FF0000E013C90E6B7
:1031D00045EA060E8DE60CEA135594EA0C0F08BF7B
:1031E00095EA0C0F3FF43BAF94EA0C0F0AD150EA7A
:1031F00001347FF434AF95EA0C0F7FF425AF10460D
:1032000019462CE795EA0C0F06D152EA03353FF434
:10321000FDAE1046194622E750EA410618BF52EAB1
:1032200043067FF4C5AE50EA41047FF40DAF52EA85
:1032300043057FF4EBAE12E74FEA410212F50012AC
:1032400015D211D56FF47873B3EB625212D94FEAED
:10325000C12343F0004343EA505311F0004F23FAD7
:1032600002F018BF404270474FF00000704750EA2C
:10327000013005D111F0004008BF6FF000407047E9
:103280004FF00000704700BF80F0004002E000BF38
:1032900081F0004142001FBF5FEA410392EA030F41
:1032A0007FEA226C7FEA236C6AD04FEA1262D2EB8B
:1032B0001363C1BFD218414048404140B8BF5B4290
:1032C000192B88BF704710F0004F40F4000020F029
:1032D0007F4018BF404211F0004F41F4000121F03F
:1032E0007F4118BF494292EA030F3FD0A2F1010289
:1032F00041FA03FC10EB0C00C3F1200301FA03F1C7
:1033000000F0004302D5494260EB4000B0F5000FE9
:1033100013D3B0F1807F06D340084FEA310102F1A8
:103320000102FE2A51D2B1F1004F40EBC25008BF5A
:1033300020F0010040EA03007047490040EB000024
:1033400010F4000FA2F10102EDD1B0FA80FCACF153
:10335000080CB2EB0C0200FA0CF0AABF00EBC25052
:1033600052421843BCBFD0401843704792F0000F40
:1033700081F4000106BF80F400000132013BB5E793
:103380004FEA41037FEA226C18BF7FEA236C21D009
:1033900092EA030F04D092F0000F08BF084670476E
:1033A00090EA010F1CBF0020704712F07F4F04D13C
:1033B000400028BF40F00040704712F100723CBF4F
:1033C00000F50000704700F0004343F0FE4040F479
:1033D000000070477FEA226216BF08467FEA236337
:1033E0000146420206BF5FEA412390EA010F40F422
:1033F000800070474FF0000304E000BF10F000436E
:1034000048BF40425FEA000C08BF704743F0964354
:1034100001464FF000001CE050EA010208BF70476F
:103420004FF000030AE000BF50EA010208BF7047F6
:1034300011F0004302D5404261EB41015FEA010C0B
:1034400002BF84460146002043F0B64308BFA3F103
:103450008053A3F50003BCFA8CF2083AA3EBC253E5
:1034600010DB01FA02FC634400FA02FCC2F1200204
:10347000BCF1004F20FA02F243EB020008BF20F03B
:103480000100704702F1200201FA02FCC2F12002A1
:1034900050EA4C0021FA02F243EB020008BF20EA96
:1034A000DC707047FDF79DFA002103E00A4B5B5882
:1034B0004350043109480A4B42189A42F6D3094A4C
:1034C00002E0002313600432074B9A42F9D300F064
:1034D0000DF8804770470000443A01000880FF1F44
:1034E0007C85FF1F0086FF1F24120020264C08B594
:1034F000F4F7C7FFF5F72EF8F5F796F9F5F7A8F901
:10350000F5F7B2F8F5F7AAFBFCF7F0FAFCF700F8CC
:10351000F5F74BFDF5F73EFA2078F5F7B5F8E078CA
:10352000F5F722F9F5F7E0FA28B1F5F7DDFA607062
:10353000F5F7DAFAA060F5F76DFB21896079228A48
:10354000FCF718F9FDF738F9FCF7E0FFFCF764FB2E
:103550000E4B4FF400725A60F7F710F8FAF79EFE20
:103560000B4B04225A60FAF7EBFAFAF733FFFAF73B
:1035700096FEF5F7EEFAF5F73DFB0028F3D0FCF7E1
:10358000C5FFF6F7FBFFEEE70C80FF1F80F00F4052
:1035900000F00F4070B4860746D0541E002A41D078
:1035A000CAB2034602E014F1FF343BD303F8012B07
:1035B0009D07F8D1032C2ED9CDB245EA05250F2C55
:1035C00045EA054519D903F110022646103E0F2E93
:1035D00042F8105C42F80C5C42F8085C42F8045C6B
:1035E00002F11002F2D8A4F1100222F00F0204F04E
:1035F0000F041032032C13440DD91E462246043A00
:10360000032A46F8045BFAD8221F22F00302043290
:10361000134404F003042CB1C9B21C4403F8011B89
:103620009C42FBD170BC704714460346C2E700BF02
:10363000024B13B1024800F005B8704700000000CB
:1036400051360100002301461A46184600F01EB804
:1036500038B50A4C0A4D641BA4100AD004F180430B
:10366000013B05EB8305013C55F804399847002CD4
:10367000F9D1BDE8384000F0D9B900BF443A0100A3
:10368000403A0100704700BF704700BF2DE9F84382
:103690002C4D0646286898460F469146FFF7F2FFE4
:1036A000294B1C68D4F84831002B3ED05A681F2A99
:1036B0001CDC02F1010E76B103EB82010124C1F89A
:1036C0008890D3F8880194402043022EC3F88801E3
:1036D000C1F8088123D00232C3F804E0286843F817
:1036E0002270FFF7D1FF0020BDE8F883174B0BB322
:1036F0004FF4C870AFF300800346D8B1D4F8482126
:103700000260002141600A46C4F848014FF0010EF2
:10371000C0F88811C0F88C11002EDCD0CCE7D3F8AB
:103720008C110C43C3F88C41D5E704F5A673C4F89B
:103730004831BBE72868FFF7A7FF4FF0FF30BDE82F
:10374000F88300BF7885FF1F1C3A010000000000CD
:103750008025000040380000004B00008070000011
:103760000096000000E10000002C010000C20100F2
:103770000084030090D0030020A1070040420F0006
:1037800000000000E0930400C0270900FF00FF00D4
:103790000000000064F00000E803000010270000B3
:1037A00010270000140000000A00000000000000C4
:1037B000FFFFFF3F00000100640000006400000004
:1037C00000070000F40100000000000000000000FD
:1037D00000000000000000000000000000000000E9
:1037E0000050C300008813000140080800000000DA
:1037F00000000000C8000000010000000080000080
:10380000000000000000000000C8000000C8000028
:1038100000000000000000000000000000000000A8
:10382000000000000000000000000000C8000001CF
:103830000000000000000000000000000000000088
:103840000000000000000000000000000000000078
:103850000000000000000000000000000000000068
:103860000001010001000000000000000000000055
:103870000000010000000000000000000000000047
:103880000101010000000000000000000001000034
:103890000000000001010100010100010100000021
:1038A0000000000000000000000000000000000018
:1038B0000000000000000000000000000000000008
:1038C00000000000000000000000010100000001F5
:1038D00000010001000000000000000000000000E6
:1038E0006580FF1F04000000090400004439010046
:1038F000543901000000000000000000000000003A
:10390000000000003C81FF1FF980FF1F0000000045
:1039100000000000000000000000000000000000A7
:103920000000120043000000000000000000000042
:103930000301020110000202001000030301100045
:10394000000100006580FF1FBF80FF1F9980FF1FDF
:103950007780FF1F043A2622D9260100D50F0100E7
:103960006D100100DD0D01000122010001220100A6
:1039700001220100012201000122010001220100B7
:1039800001220100012201000122010001220100A7
:1039900001220100012201005F130100F512010064
:1039A0005513010021130100F5120100012201004D
:1039B000E1120100CD1301009D24010069250100E1
:1039C0000000000069250100000000005D240100E6
:1039D0008524010000000000C5230100F52301003B
:1039E0005D2601003D26010099230100010100012F
:1039F00001000000000101000000000001010101C0
:103A000001000000010100010100010000010000AF
:103A10000100003333313256313131005081FF1F04
:103A2000F8B500BFF8BC08BC9E467047F8B500BFAB
:083A3000F8BC08BC9E4670477B
:083A3800313601003584000065
:043A400011840000ED
:103A4400133A010000010200000800000100000018
:103A54000200000000000000000000000000000060
:103A64000000000000000000000000000000000052
:103A74000000000000000000000000000000000042
:103A840000000000000103040506071701000200FE
:103A94000400A1200000000002000000FF0403094C
:103AA4000400C20100000008000000000000002221
:103AB40003420041004400200053005400520049D6
:103AC400004E004700200049004E004400450058C5
:103AD40000260353007400650070007000650072D6
:103AE4000020004D006F0074006F0072002000443D
:103AF400006500760020003A035400520049004E4D
:103B04000041004D004900430020004D006F007447
:103B14000069006F006E00200043006F006E0074A7
:103B24000072006F006C00200020002000200020A4
:103B34000009024300020100C0320904000001022E
:103B440002000005240010010524010101042402DF
:103B54000605240600010705830310000A09040171
:103B640000020A0000000705810210000007050298
:103B74000210000012010002020000103C2A0001A1
:103B84000200010200010000000000003C84FF1F4D
:103B9400A484FF1F0C85FF1F00000000000000002C
:103BA4000000000000000000000000000000000011
:103BB4000000000000000000000000000000000001
:103BC40000000000000000000000000000000000F1
:103BD40000000000000000000000000000000000E1
:103BE40000000000000000000000000000000000D1
:103BF40000000000000000000000000000000000C1
:103C040000000000000000000000000000000000B0
:103C140000000000000000000000000000000000A0
:103C24000000000000000000000000000000000090
:103C340001000000000000000E33CDAB34126DE62D
:103C4400ECDE05000B000000000000000000000096
:103C54000000000000000000000000000000000060
:103C64000000000000000000000000000000000050
:103C74000000000000000000000000000000000040
:103C84000000000000000000000000000000000030
:043FB40000120020D7
:103FB800443A01000880FF1F74050000000000005B
:083FC8000000000000000000F1
:04000003100034A510
:00000001FF
